:020000040002F8
:10600000E0600020010D030083740200B3760200FB
:1060100057780200F778020027790200000000009C
:10602000000000000000000000000000637A020091
:106030009F7A020000000000C37A0200A77B0200E2
:1060400085F70200EF7D020069DF02003B7E02005F
:106050004F910200579102003DF40200FF910200AF
:10606000EB9D020013A102001FB002007FBF0200DF
:1060700033C002004BD1020003D20200A7E50200A8
:10608000FFEC020091BD02008BFF020069070300D4
:10609000AF080300BF08030071B20200D70A030073
:1060A0006F0F0300AD0F0300AF0F0300B10F03002C
:1060B000B30F0300B50F0300000000000000000054
:1060C000B70F0300B90F0300BB0F0300BD0F0300A0
:1060D000BF0F0300C10F0300C30F03000000000047
:1060E00000000000000000000000000000000000B0
:1060F00000000000000000000000000000000000A0
:10610000000000000000000000000000000000008F
:10611000000000000000000000000000000000007F
:10612000000000000000000000000000000000006F
:10613000000000000000000000000000000000005F
:10614000000000000000000000000000000000004F
:10615000000000000000000000000000000000003F
:10616000000000000000000000000000000000002F
:10617000000000000000000000000000000000001F
:10618000000000000000000000000000000000000F
:1061900000000000000000000000000000000000FF
:1061A00000000000000000000000000000000000EF
:1061B00000000000000000000000000000000000DF
:1061C00000000000000000000000000000000000CF
:1061D00000000000000000000000000000000000BF
:1061E00000000000000000000000000000000000AF
:1061F000000000000000000000000000000000009F
:106200002DE9F84F74A7A2B0D7E90045CDE90045C4
:106210002C9EDFF8307C04918DF843605FF0000124
:106220006FA40D9112944FF0FF3682469046994626
:106230000FE0C3462C461BF8011B0498D0470028EA
:10624000049000F0B2800D98401C641E0D90F2D1B5
:10625000A84498F80000252807D10021079108914B
:1062600009910A910B910C910DE06A463146404626
:1062700001F01DF8050001D10D98B5E0D9D5012533
:10628000E6E741F0010118F8010F2028F9D0232892
:106290000CD02B2804D02D2805D0302809D086E03A
:1062A00041F00201EFE741F00401ECE741F00801A1
:1062B000E9E741F01001E6E700200F900AE00F98AF
:1062C000B84205DA00EB800302EB4302303A0F924A
:1062D00008F1010898F80020A2F130000A28EED356
:1062E00098F800002E2818BF0E9629D118F8010F33
:1062F0002A280BD1D9F80000C9F8000008F10108DC
:1063000050F8042BC9F800000E9219E02D280CBF9C
:1063100018F8010B002000220E920BE040B90E9AF3
:10632000BA4205DA02EB820403EB4403303B0E93DE
:1063300008F1010898F80030A3F130020A2AEDD3E1
:10634000ADF84010129898F8001000F0BBFF08B1AB
:1063500018F8010B8DF842009DF84200682804BF30
:1063600098F80010682903D162208DF8420008E0F7
:106370006C2804BF98F800006C2804D171218DF8B6
:10638000421008F1010813A806904A4618F8013B8C
:1063900002A9504600F068F838B913AA02A950467D
:1063A00000F0CAF900287FF554AF30461CE02A28D7
:1063B00082D1D9F80020C9F8002052F8040BC9F89E
:1063C000002000280F9003D540420F9041F00401B7
:1063D00008F1010884E70000000000000000000050
:1063E000686A6C747A4C000023B0BDE8F08F6228B4
:1063F00020D0682811D06A2803D06C2827D07128B3
:1064000025D10868C01D20F007000860D0E90023EE
:1064100008300860194610467047002A0A680A606A
:10642000106803D0121D0A6000B217E0121D0A6046
:1064300080B217E0002A0A680A60106803D0121DB3
:106440000A6040B20AE0121D0A60C0B20AE0002AE7
:106450000A680A60106803D0121D0A60C1177047ED
:10646000121D0A60002170477CB50D4611461C467E
:106470002E69B4F1250200F04D811C3A00F08680AF
:10648000121F022A40F282800E3A00F00781521F4A
:106490005AD0093A7AD0921E16D0521E35D0521ECA
:1064A000022A73D9121F30D0521F00F09A80521E58
:1064B0004AD0521E00F0E480D21E00F0FD80921EF1
:1064C00042D0D21E40D02BE195F83A206C2A09D058
:1064D0006869421C6A610A680A6052F8043B0A60F3
:1064E000335427E10A680A6052F8043B0A6000212D
:1064F000009301914FF0FF322A6329466A4600F06B
:1065000096F9002840F1168101E195F83A00012240
:10651000FFF76DFFC5E900010023994204DA6869BD
:10652000411C69612D210DE0288F810704D5686920
:10653000411C69612B2105E0C00722D56869411C17
:106540006961202131541CE095F83A000022FFF7E0
:106550004EFFC5E9000195F83800010711D5D5E9CE
:1065600000230020834208BF82420AD044F020006A
:10657000782806D1686930213154401C411C69617A
:106580003454214668693044E86083E00868C01DDF
:1065900020F007000860D0E9002308300860C5E952
:1065A0000023D5E90001C80F04D06869411C696166
:1065B0002D210DE0288F810704D56869411C696190
:1065C0002B2105E0C00704D56869411C69612021C1
:1065D000315468693044E8602146284600F032FAB8
:1065E000A8E005F13A02507820B14FF0FF340FF6E1
:1065F000243070E01078622808D0682824D06A28F7
:1066000012D06C282ED071280ED02BE00A680A60B8
:1066100052F8040B0A6020B94FF0FF340FF60C302B
:1066200059E0E96A017085E00A680A6052F8040BD3
:106630000A6020B94FF0FF340FF6F0204BE0EA6A11
:10664000D317C0E9002375E00A680A6052F8040B0A
:106650000A6020B94FF0FF340FF6D0203BE0E96A22
:10666000018067E00A680A6052F8040B0A6020B9EA
:106670004FF0FF340FF6B4202DE0E96A016059E0D5
:106680000A680A6052F8040B0A600021C5E900019B
:10669000EE607821284600F029F94BE06C2285F85D
:1066A0003A200B680B6053F8042B0B6052BB4FF081
:1066B000FF340FF6AC200EE095F83A206C2AF0D0AB
:1066C0000868086050F8044B0860EC603CB94FF073
:1066D000FF340FF6702000F00FFE201A76BD2E6BEF
:1066E000002E04D5204600F027FE044608E032467E
:1066F0000021204600F040FE002814BF041B344651
:10670000AC6117E0294600F092F8002812D54FF04E
:10671000FF3076BD6869411C69612521315409E06B
:106720006969481C686125227254210002D0411C0D
:1067300069613454002076BD2DE9F0410E460546CE
:10674000716B7069B46A091A306A091AB069091A5A
:10675000706A091AF069091A96F838000C1B41078B
:1067600090460DD4002C0BDD2746B0682021A847A9
:106770000028B06057D0F06A401C7F1EF062F4D150
:10678000736942463146284600F0ACFC00284AD1E5
:10679000376A002F0ADDB0683021A8470028B060B2
:1067A00041D0F06A401C7F1EF062F4D1B369F268F8
:1067B0003146284600F096FCA8BB776A002F09DD19
:1067C000B0683021A847B06068B3F06A401C7F1EF3
:1067D000F062F5D1F068B169F36942183146284694
:1067E00000F080FCF8B9B76A002F09DDB0683021ED
:1067F000A847B060B8B1F06A401C7F1EF062F5D1C6
:1068000096F8380041070BD5002C09DDB06820212F
:10681000A847B06038B1F06A401C641EF062F5D140
:106820000020BDE8F0814FF0FF30BDE8F0812DE998
:10683000F8470D46A3B02F6B002F8146904648BF06
:106840006FF0004700F0C4FD696B40180FF62C1183
:106850008128D1E90023CDE9012328BF4FF0FF3083
:106860003ED20024002F2FDDD8F8001001AA684680
:1068700000F01FFD0646002E35D4D8F8000008B9F8
:10688000761E30D4B7421FDB6869301881280AD3DE
:106890000020686303AA29464846FFF74DFF04001D
:1068A00012D40020686103A8D5F814A032466946C6
:1068B000504400F093FDB244C5F814A058F8040BFE
:1068C000002818BFBF1BCDD12CB903AA29464846C2
:1068D000FFF732FF044614B9002068616863204660
:1068E00024B0BDE8F0874FF0FF34F8E72DE9FC470E
:1068F00007468A463E69BAF16F0F08BF082405D0E3
:106900004AF02001782914BF0A2410243C25D7E935
:106910000023BAF1640F18BFBAF1690F9046994687
:1069200006D100218B4203DAD8F1000869EB49094E
:106930000020814508BF80451FD1386BE8B9082C7D
:106940004CD197F83800010748D530203B2586F810
:106950003B0043E000280ED597F8380000F0140003
:10696000102808D17A6B7869121A386A121A511AEB
:106970000029C8BF3962BDE8F3878DF800A0404602
:1069800049462246E31700F07DFD3032D0B26D1E3D
:106990003A28019504DB9DF80000A0F151018A1806
:1069A0007255404649462246E31700F06BFD80468B
:1069B00089460020814508BF804503D0F8687119D9
:1069C0008842DCD3082C09D197F83800010705D597
:1069D000715D302902D06D1E30207055C5F13C012B
:1069E000B9617019F860386B8142B3DA411A3962C3
:1069F0004FF6EF70398F01403987BDE8F3872DE9F5
:106A0000D04306460F4614464FF00008DFF838948E
:106A100012E0E00707D542464B463046394600F0C3
:106A200049FE06460F464046494642464B4600F060
:106A300041FE641080468946002CEAD13046394632
:106A4000BDE8D0832DE9F34F054641F020048DB019
:106A5000D5E90089612C02AE09D0286B002848BF17
:106A6000062003D408BF672C01D101202863D5E993
:106A7000002358004015401C0ED119030CD00320F0
:106A8000A8619DF8380061381A2802D20FF2F4612B
:106A900011E00FF2F4610EE058004015401C0FD1D8
:106AA00019030DD10320A8619DF8380061381A2818
:106AB00014D30FF2DC61E868032200F08FFCD3E10D
:106AC000194621F00043B3F5801F10460DD2002770
:106AD000BB4208BFBA42019703D111E00FF2AC618B
:106AE000E9E701AA00F0B8FE0AE0DFF8607307EBFF
:106AF0001352DFF85C3301921940DFF85833194321
:106B0000C5E90001612C0ED1E86830210170811CBB
:106B1000E9609DF8381061290CBF78215821417037
:106B20006869801C6861D5E900AB2BF00043002048
:106B30002AF00002834204BF8242002300F05A81FF
:106B4000612C40F0A980286B00284CBF2120401CFC
:106B500000904046009F7F1C49460022002300F021
:106B6000B3FED94601988DF8082038BF89F0004956
:106B7000001F0190002FD0460DF1090040F349811C
:106B800040F2FF71DFF8D0B20C910646404649460C
:106B90000022002300F0B0FE80F03A814800400D52
:106BA00000F11C0210D0002A0EDD0C98824205DB99
:106BB00009F0004040EA0B01002013E0A44808401F
:106BC00040EA025140460DE029F00043002028F041
:106BD0000002834208BF82420FBF40461C2240464B
:106BE00000F0A2FE8046894600F03CFFFF1F002F08
:106BF000044609DD00F054FF02460B464046494674
:106C000000F060FF80468946F01D072104E004F093
:106C10000F0200F8012D2411002C01DD491EF6D5CC
:106C2000491E5CBF002200F8012DF9D5ECE00020E0
:106C3000194602AA0A4400E05B1E12F80149491EE7
:106C40008442F9D00F2804D10DF10900425C521C96
:106C50004254002904D50198001D02AE5B1C01902E
:106C6000591E12D49DF838007218147804F13008B7
:106C70005FFA88F4392CC4BFA0F13A04A044491E3D
:106C800002F80189F1D58DF83800286B002840F111
:106C9000B080591E2963ACE04046494600220023DB
:106CA00000F012FE019938BF89F0004947F2975071
:106CB00041436A4A91FBF2F20192D2F1070204DDEC
:106CC00040464946FFF79BFE0AE0524200206449D5
:106CD000FFF795FE02460B464046494600F064FF2A
:106CE0008046662C286BDFF87CB106BF019F0A370F
:106CF00006273F18142FC8BF142730208DF808002E
:106D000089460DF1090000E03046002F34DD0646CB
:106D10004046494601F06CF801460A4606F1080370
:106D200004200A26B2FBF6F606EB860EA2EB4E0214
:106D3000303203F8012C0A22B6FBF2F202EB820E8B
:106D4000A6EB4E063036401E03F8026DE9D1083F2F
:106D5000002F03F10806D7DD084601F05DF8024672
:106D60000B464046494600F0ADFE00225B4600F06F
:106D7000A1FC80468946CBE70DF10901401A0DF1CF
:106D8000090604E00199491E401E0191761C3178E4
:106D90003029F7D0662C02D10199491C03E0652CFB
:106DA0000CBF012100212B6BCB189842B8BF431EAA
:106DB000002B1ED4834204DAF05C3528A8BF3920AA
:106DC00000DA30201946721E02EB010800E05B1E5B
:106DD00018F80199491E8145F9D0392802D1705C13
:106DE000401C7054002904D50198401C16465B1CB9
:106DF0000190019800B200901BB29DF83810324605
:106E0000284600F035F82FE0C61D002F3FF7BEAE34
:106E100030460DF10901401A009903468842C8BF67
:106E20000B46002B0DF109063FF52FAF8342BFF64D
:106E3000FEAE0DF10900C05C07287FF7F8AE0F2009
:106E4000F6E60000CBCCCC0C0000244002FCFFFF97
:106E5000FFFF0F800000E03F0000F07FA0860100F0
:106E60000000F03F84D797410FB0BDE8F08F0000DD
:106E70002DE9F84783B006468A461746984600F043
:106E80001AFAB8F1000F406A356B90F8009002DCF6
:106E90004FF00108BFA7BDF930404AF02000662836
:106EA00008BF641C15D0672840F0848014F1040FDB
:106EB000C0F28680AC4280F2838096F83800641C71
:106EC000010702D4A845B8BF454620B22D1A48BFD5
:106ED00000250FFA84FAF068B169BAF1000F25DCD9
:106EE0004A1C30234354002D03DC96F83800010778
:106EF00003D5F06800F80290521C15EB0A0FB8BFDA
:106F00006C4220B2441941424445B8BFA046B26128
:106F100071620FFA88F5F561F068B3692A4639465F
:106F2000184400F05BFA641BB462C4E022B29045DE
:106F3000084417DA4246394600F050FAB069404436
:106F4000B061AAEB0801002D716203DC96F83810DD
:106F50000A0705D5F16801F80090F069401CF0615E
:106F6000B562A8E0394600F039FAB069002D504406
:106F7000A8EB040803DC96F838100A0703D5F1687B
:106F800001F80090401CB0610FFA88F08542F0686B
:106F9000B369B8BFA8460FFA88F207EB0A01184494
:106FA00000F01CFAB0690FFA88F10844B061681A61
:106FB000706280E0BAF1610F14D14FF0700A16E0F0
:106FC000A84504DA96F838100A0758BF45466D1EE2
:106FD00048BF0025BAF1670F14BF4FF0450A4FF0C4
:106FE000650A04E0BAF1410F08BF4FF0500AB169D9
:106FF000F368481CB061002D17F8012B5A5403DCCC
:1070000096F838100A071BD5F168431CB36101F8E4
:107010000090002D14DDA8F101080FFA88F08542D8
:10702000F068B8BFA8460FFA88F23946184400F055
:10703000D5F9B0690FFA88F108446D1AB06175622C
:10704000F068B1690844002C80F800A003D42B211B
:107050004170811C03E02D2141706442811C00209D
:107060006A460AE023460A2493FBF4F404EB840501
:10707000A3EB450302F8013B401C24B2002CF1DCD9
:10708000012806DC4AF02002652A04BF302201F8FC
:10709000012B48B9302001F8010B07E0401E1DF814
:1070A0000020303201F8012B0028F7DCF068B269CB
:1070B0001044091AF16196F8380000F01400102805
:1070C0000DD17169B0694118706A4118F0694118B1
:1070D000B06A4118706B8142BCBF411A316204B082
:1070E000BDE8F087F8B505460E4617461C46002059
:1070F00074B117F8011BB068A847B06030B1F06AEE
:10710000401CF0620020641EF3D1F2BD4FF0FF304E
:10711000F2BD00007072696E74665F733A20256E6E
:1071200020646973616C6C6F776564007072696E5E
:1071300074663A2062616420256E20617267756D05
:10714000656E74007072696E74665F733A20626176
:107150006420257320617267756D656E7400000090
:107160007072696E74665F733A2062616420256C88
:107170007320617267756D656E7400000000000019
:10718000000000006E616E004E414E00696E6600A8
:10719000494E46003000F0B4024610689568131856
:1071A000506803EB5004C00721D54D441FE0F0BCEC
:1071B00002F10C00704713F8017B05F8017B491EB2
:1071C000F9D1A0B1B60813F8011B06F00306032E8F
:1071D00008BF13F8016B01EB06214942801C2944CA
:1071E00005D011F8016B05F8016B401EF9D1A342DF
:1071F000DDD013F8016B16F0030104BF13F8011B77
:10720000C91C30090F28DAD113F8010B0F30D6E76B
:10721000613807E005E0A0F161011A2901D20120DF
:10722000704741381A288041C00F7047A0F12101F2
:107230000F290AD3A0F13A02062A06D9A0F15B0170
:10724000062902D37B380428EDE7012070471B484C
:10725000704730B45368D418042B09DA41B105786B
:1072600004F8015B10F8015B15B15B1C491EF3E7E4
:10727000536030BC704738B514461D4661B1FFF706
:10728000E8FF61686A6B204690476FF00102811A3F
:1072900002D0491E03D005E06FF0010032BD4FF06F
:1072A000FF3032BD0021616032BDDA6B1047034B05
:1072B000E1E7024BF9E70248704700005C2C002030
:1072C000242C00200278C9B28A421AB11CBF10F8DF
:1072D000012FF9E718BF00207047B1F5807F02D376
:1072E0004FF0FF3070470170012070470078401E5A
:1072F0008041C043C00F704780B500B906A0054962
:107300000B681BB122220021984701E000F091FD9B
:10731000222002BDC8400020636F6E7374726169E1
:107320006E742068616E646C65723A2062616420DC
:107330006D6573736167650000F10103810704D017
:1073400010F8011B89B18107FAD10268B2F101314D
:10735000914311F0803F04BF50F8042FF6E710F876
:10736000011B11B110F8011BFBE7C01A704702683E
:10737000531C036011707047C9B2830706D0521EB8
:1073800022D310F8013B9942F7D11FE0083A13D3FA
:1073900002F1040241EA012141EA014150F8043BB3
:1073A000121F21BF4B40A3F1013C2CEA030C1CF03F
:1073B000803FF3D0C9B2001F083210F8013B521EC3
:1073C00028BF91EA030FF8D818BF0120401E70476C
:1073D00080B5FFF73CFF006C02BD000062B38B0775
:1073E00008D0521E11F8013B00F8013B00F0248048
:1073F0008B07F6D1830740F0208000BF103A07D3F7
:1074000030B4B1E83810103AA0E83810F9D230BCE6
:10741000530724BFB1E80810A0E8081044BF51F892
:10742000043B40F8043BD20724BF31F8022B20F87C
:10743000022B44BF0B7803707047121F17D35B00F9
:1074400009D151F8043B20F8023B1B0C121F20F815
:10745000023BF6D20BE051F8043B00F8013B1B0A5B
:1074600020F8023B1B0C121F00F8013BF3D238BF7F
:10747000121D521E24BF11F8013B00F8013BF8D841
:107480007047FEE7B3BBD9B1B2F5803F7DD2022A87
:107490001ED98C46B1FBF2F102FB11C31B0443EA77
:1074A0001043B3FBF2FC02FB1C3380B240EA0343FF
:1074B000B3FBF2F002FB103240EA0C4000237047AD
:1074C000022A05D98446B0FBF2F002FB10C27047D5
:1074D0004AB105D100F0010249085FEA3000704767
:1074E00000220023704700F0A7BC0B00020000211F
:1074F00000207047904271EB030CF6D3B3F5803F48
:107500002FD2F0B5B3FA83F7B1FA81F4A7F10F0ED9
:107510003D1B5340CEF1200602FA0EF2F3415340D8
:10752000B5F10F0746D80F3C2C444140C4F120066A
:10753000A040F1414140B1FBF3F603FB1611A2FB61
:107540000645001BA94102D2761E8018594180EAE7
:10755000010221FA0EF362FA0EF200215A4030467F
:10756000F0BD30B4B1FBF3FC03FB1C11A2FB0C45D6
:10757000001BA94103D2ACF1010C8018594130BC69
:1075800002460B46604600217047B2F1807F65D30A
:10759000F0B5B2FA82F7B1FA81F4C7F10F063D1BDC
:1075A00022FA06F307F1110EF24120355A40B5F1E7
:1075B0000F07B8D94140C4F12006A040F141414035
:1075C000B1FBF3FC03FB1C11A2FB0C45001BA94102
:1075D00003D2BCF1010C801859410F2F12D30F3F79
:1075E000C90341EA5041B1FBF3F603FB1611A2FBBC
:1075F0000645D4EBC030A94102D2761E801859410D
:1076000046EACC3C07B34140C7F12006B840F141FF
:107610004140B1FBF3F603FB1611A2FB0645001B2C
:10762000A94102D2761E8018594180EA010221FA4E
:107630000EF3C7F1200462FA0EF20CFA07F05A407A
:107640002CFA04F13043F0BD80EA010221FA0EF376
:10765000002162FA0EF260465A40F0BD8C46B1FB42
:10766000F2F102FB11C31B0243EA1063B3FBF2FC0D
:1076700002FB1C331B024CEA002043EA1063B3FBFD
:10768000F2FC02FB1C331B024CEA002043EA1063AD
:10769000B3FBF2FC02FB1C331B024CEA002043EA62
:1076A0001063B3FBF2FC02FB1C324CEA0020002307
:1076B0007047FEE7B0B581EA030C0CF0004C40F2D5
:1076C000FF7515EA11541DBF15EA1357AC42AF42BE
:1076D00039E0E41923EA455343F48013C90241F029
:1076E000004141EA505EC7021100A7FB02020028D8
:1076F0004FF00000EEFB01204FF00001E3FB0721FB
:1077000018BF42F00102401800214941E3FB0E017D
:10771000A4F580640F0302D252004041494154F164
:1077200001046CDD470872F1004250F1000051EB9A
:107730000451A1F580115CBF41EA0C01B0BD4CEAD7
:1077400005510020B0BD05EA1357AC4214BFAF424B
:1077500041E050EA410E1CBF52EA430E02E061468E
:107760000020B0BD24423C441BD15FEA070EF6D096
:10777000090302BF01460020AEF1140EB1FA81F7F1
:10778000AEEB070401FA07FE0C37C7F1200100FA3F
:1077900007F7C8404EEA000E23EA455343F480132E
:1077A000A2E733F00043B3FA83F704BFB2FA82FED4
:1077B00077440B3FE41BB7F1200E2FBF02FA0EF304
:1077C000BB40C7F1200E22FA0EFE38BF43EA0E037B
:1077D000BA40641C82E750EA410E14BF52EA430EDD
:1077E0006FF000014FF4001717EB430F8ABF1946E3
:1077F00017EB410FB5E74CEA05510020B0BDD4F1BD
:107800000104B4F120070FDAC4F12007520828BFA1
:1078100042F0010210FA07F501FA07F7E1BF2A4327
:10782000E0403843E1400FE0352C98DCC7F12004FC
:1078300052EA400220FA07F218BF42F0010231FA80
:1078400007F0A1400A43002172F1004250F100000C
:1078500051EB0C01B0BDFEE710B5144600F002F884
:10786000226010BDC1F30A5343B14A0012F5001F54
:1078700028D2A3F2FE32A1EB0251704750EA410C2C
:1078800020D001F0004C31EA0C01B1FA81F204BFC2
:10789000B0FA80F3D2180B3AB2F120032CBF00FAF1
:1078A00003F1914041EA0C013EBFC2F1200C20FAE5
:1078B0000CF319439040524240F2FD33D21A01EBCF
:1078C00003517047002270474FF4001C1CEB410F1E
:1078D00094BF1CEB430F09E041EA030C50EA4C0C47
:1078E00052EA0C0C03D2994208BF9042704714BF71
:1078F0008B4282427047FEE74FF4001C1CEB410FA5
:1079000094BF1CEB430F09E041EA030C50EA4C0C16
:1079100052EA0C0C03D28B4208BF8242704714BF5C
:10792000994290427047FEE7124254D440F2FF7CE5
:107930001CEA11530FD0634531D09B1863453CBFFF
:1079400001EB0251704701F0004141EA0C51002067
:10795000AFF30080704750EA410320D001F0004CA3
:1079600091EA0C011CD0B1FA81F30B3B9A420DD97C
:10797000D21A994051EA0C01C3F1200C20FA0CFCF8
:1079800061449840531C40F2FF7CD7E7914041EAA4
:107990000C01C2F1200C20FA0CF3194390407047FF
:1079A000B0FA80F31533202BE0D3202AEED3203A0F
:1079B000203B9A4209D9D21A00FA03F141EA0C019C
:1079C0000020531C40F2FF7CB8E700FA02F141EAC4
:1079D0000C0100207047524240F2FF7C1CEA115318
:1079E0000DD06345DBD0B2EB030C3CBFA1EB0251E1
:1079F00070470CF1010221EA035141F4801150EA71
:107A0000410CCCD001F0004C352A27DC30B481EA9F
:107A10000C01B2F1200309DAC2F12003044601FA95
:107A200003F5D0402843D1409C400CE0C3F1200234
:107A3000450020FA03F418BF44F0010421FA03F0D2
:107A400091400C43002174F1004550F1000051EBCE
:107A50000C01244230BC7FF47BAF704761460020AC
:107A600076E7FEE7C1F30A5340F2FE329B1A14DDBB
:107A7000D3F120034FEAE17208DDC90241EA505117
:107A800041F00040D84080185040704703F2E13088
:107A900010B1D24382F00040704700207047FEE7EB
:107AA000C11768B14840401AB0FA80F29040D21C29
:107AB000C907C2F5846241EA025202EBD0214005B7
:107AC0007047FEE770B44FF0004591EA030F40F1B4
:107AD000B5816B40841A71EB030603D2001BB141E0
:107AE000121973414FF4001C1CEB410F34BF7CEBA7
:107AF000430442E00C0DA4EB1356352E4FDC45EA4F
:107B0000C323DB0A45EAC121C912B6F120050DDD08
:107B100063FA05F6EB4086EA0305124218BF45F00A
:107B20000105C01851F100010CD213E062FA06F50C
:107B3000F2405540F3415A40B340F3405A40801858
:107B4000594107D349085FEA30005FEA350528BF8D
:107B500045F0010501F58011420875F1004250F130
:107B6000000041EB04514E0016F5001F70BC38BFF9
:107B700070470020090D090570471CEB410F10D21A
:107B800052EA43060BD0BCEB410F05D80C0DAB43BA
:107B9000661E342EB6DD02E0AB438018594170BC3E
:107BA000704770BC7047FEE7F0B540F2FF7581EAA0
:107BB000030C0CF0004C15EA11541DBF15EA1357C5
:107BC000AC42AF42E5E0BC41C1F31301C3F3130380
:107BD000801A994143F4801304D2641E4000494145
:107BE00080185941C90241EA5051B1FBF3F603FB39
:107BF0001611A2FB0675D7EBC020A94102D2761E52
:107C000080185941C90241EA5051B1FBF3FE03FB10
:107C10001E11A2FB0E75D7EBC020A94103D2AEF115
:107C2000010E80185941890241EA9051760546EAD1
:107C30008E2EB1FBF3F603FB1611A2FB0675D7EBF4
:107C40008020A94102D2761E80185941C90241EA1A
:107C500050514EEA060EB1FBF3F603FB1611A2FBE0
:107C60000675D7EBC020A94102D2761E8018594173
:107C7000C90241EA5051B1FBF3F703FB1711A2FB14
:107C80000735D3EBC020A94167F100070CBF0042C4
:107C900047F0010766F3D5274FEA1E31B80814F5FF
:107CA000806412DDBD0775F1004250EB0E5051EBC0
:107CB000045111F5801F5CBF41EA0C01F0BD4CF08E
:107CC0007F6141F0E0410020F0BDBD076D0840EA52
:107CD0000E5041F48011D4F10104B4F120060ADA07
:107CE000C4F120060200E04001FA06F3E140184327
:107CF000B24015430EE0342C13DCC6F1200445EAF3
:107D000040056D0820FA06F2154321FA06F0A1405D
:107D10000D43002175F1004250F1000051EB0C01C0
:107D2000F0BD00205FEA0C01F0BDCFB992185B41B5
:107D3000B3FA83F704BFB2FA82F6BF190B3FB7F16B
:107D400020062FBF02FA06F3BB40C7F1200622FA35
:107D500006F638BF3343BA401CB1E419641E33E75A
:107D60007F4231F00041B1FA81F404BFB0FA80F6ED
:107D7000A4190B3CB4F120062FBF00FA06F1A14074
:107D8000C4F1200620FA06F638BF3143A0403C1B60
:107D90001AE7AC421ABF05EA1357AF4212E050EAA5
:107DA00041061CBF52EA4306BFE750EA410730468E
:107DB00061461CBF41EA0551F0BD52EA430C08BFC1
:107DC000C143F0BD00204FF4001616EB410F98BFE1
:107DD00016EB430F08BF16EB410F24BFC14305E06C
:107DE00016EB430F0CBF61464CEA0551F0BDFEE7B0
:107DF000400D491840EA81200CD2490DA1F580615F
:107E0000491C40F0004005DBD1F11F0154BFC840C0
:107E1000C017704700207047014648B1B0FA80F1A2
:107E20008840C91CC1F58461090501EBD0214005DA
:107E30007047012000F0B6B87047FEE7841A71EB76
:107E4000030604D26E40001BB141121973414FF476
:107E5000001C1CEB410F34BF7CEB430682E00C0D91
:107E6000A4EB1356362E7BDC012E45EAC32341DCFE
:107E700043EA525312BFD20292025B08240545EA3C
:107E8000C12141EA5051D2EBC020994125D407D1FC
:107E9000B0FA80F610FA06F162D00020203608E031
:107EA000B1FA81F6B140C6F1200220FA02F2114384
:107EB000B0404FEAF474B4EB465434F001064FEA94
:107EC00074040AD8D6F50016760D04F00044F0408C
:107ED00061FA06F25040F1404840C00A40EA415081
:107EE00021F0004128BF5FEA500550F1000044EB4B
:107EF000D12135E0DB0A45EAC121C90AB6F12005E6
:107F00000EDD42EA0242120CC5F1200603FA06F623
:107F1000EB4042EA06056D42984161F100010DE037
:107F200062FA06F5F240554063FA06FC82EA0C025A
:107F3000F3405A406D42904161EB030111F4801F00
:107F400005D1641E620502D06D004041494121F413
:107F50008011430875F1004350F1000041EB0451DA
:107F600070BC70471CEB410F15D223F0004352EA5E
:107F700043060BD04FEA4C0CBCEB410F04D80C0D60
:107F8000661E342EB7DDEBE7801A994150EA4106B0
:107F900008BF0021E4E708BF1CEB430F28BF6FF0C8
:107FA0000001DDE780B5AFF30080024A1100182020
:107FB000ABBEFBE726000200BFF34F8FDFF8C80A15
:107FC000016811F4E061DFF860070143DFF8B80AE7
:107FD0000160BFF34F8F00BFFDE780B5002806D0DA
:107FE000DFF8A82A52F0010240214843904701BD22
:107FF00010B50400002C06D04FF47A70FFF7EDFFA7
:10800000641E002CF8D110BD80B5FFF795F9801CD7
:10801000032190FBF1F0800002BD2DE9F84304003C
:1080200088461500994600260027002C01D0002D17
:1080300001D1002074E02000FFF7E6FF814531DA2E
:1080400000206DE0DFF8480AA15D8910405CE8552A
:108050007F1CDFF83C0AA15D090111F0300104EB3F
:108060000602527851EA2211405CE8557F1CDFF885
:10807000200A04EB06014978890011F03C0104EB69
:108080000602927851EAA211405CE8557F1CDFF8A5
:10809000000A04EB0601897811F03F01405CE855C5
:1080A0007F1CF61CB8F10200864202DA381D8145B9
:1080B000C8DA464533DADFF8D809A15D8910405C9B
:1080C000E8557F1CB8F1010846450CD1DFF8C0091E
:1080D000A15D11F003010901405CE8557F1C3D20C2
:1080E000E8557F1C18E0DFF8A809A15D090111F02F
:1080F000300104EB0602527851EA2211405CE85547
:108100007F1CDFF88C0904EB0601497811F00F01A0
:1081100010F82100E8557F1C3D20E8557F1C3800F1
:10812000BDE8F28380B500F08EFF002801D000F09A
:10813000FFFF01BD18B5C3B001208DF800009DF808
:10814000000010F00F0050F010008DF8000003A8A0
:108150004FF4807100F0FCFFDFF8CC3ADFF8CC2A56
:10816000DFF8CC1A03A800F0F7FF03A8FFF7E4F844
:10817000202800DB1F20020092B203A968467CDFA2
:10818000002801D000F0D4FF0821002201AC20001B
:1081900001F002F81020ADF804003C20ADF8060014
:1081A0000020ADF808004FF4C870ADF80A0001A82F
:1081B0007ADF002801D000F0BBFF44B010BD80B5CD
:1081C00000F0B6FF01BD2DE9F8430500287800282E
:1081D00040F03F81A88A072820DB286900784128E1
:1081E0001CD1286940786E2818D1286980786428C5
:1081F00014D12869C078722810D1286900796F28B5
:108200000CD128694079692808D1286980796428C7
:1082100004D1DFF8200A00F0F3FF1AE1A88A082849
:10822000C0F2E78028690078532840F0E28028698E
:108230004078452840F0DD8028698078542840F057
:10824000D880286980793A2840F0D3802869C0789E
:10825000442823D12869007945281FD1286940790D
:1082600056281BD1AC8AE41F392C00DB382440216E
:108270000022DFF8B869300000F08EFF002006E031
:1082800029690144C979DFF8A4291154401CA0428E
:10829000F6DB0120DFF8A0190870AAE02869C07891
:1082A000542825D1286900794F2821D1286940799F
:1082B00050281DD1AC8AE41F392C00DB3824402122
:1082C0000022DFF86469300000F066FF002008E05B
:1082D00029690144C979DFF85429024482F8401021
:1082E000401CA042F4DB0120DFF84C19087080E04C
:1082F0002869C07841287CD1286900794C2878D138
:10830000286940794C2874D1A88AC01F00215FF0E9
:108310000008002700240026002210E003290DD1C8
:10832000D41BB4EB0804A41EAE8AB61AF61F761E40
:1083300004E00229F2D1B2EB08077F1E521C8242F0
:1083400009DA2B691344DB793B2BF7D1491C01294E
:10835000EFD19046F2E703294BD140210022DFF80C
:10836000C898484600F018FF20210022DFF8CC987A
:10837000484600F011FF20210022DFF8C49848464B
:1083800000F00AFF40210022DFF8A098484600F0E4
:1083900003FF42462869C11DDFF890984846FFF761
:1083A0001DF83A002869404410F10801DFF8789878
:1083B0004846FFF713F82200286917EB0801084424
:1083C00010F10901DFF874984846FFF707F832000A
:1083D000286917EB080814EB0808404410F10A015B
:1083E000DFF85C482000FEF7F9FF0120DFF84818AD
:1083F000087000261EE02869805D01F031F8040055
:10840000002C14D0112C12D02200DFF83818DFF81D
:108410003808DFF83838C01AC008000450F00100EE
:1084200001F04BFA2000002801D000F081FE112C51
:10843000E1D0761CA88A8642DDD32869A98A08443F
:1084400010F8010C0D2804D10A2001F009F81128B8
:10845000FAD0BDE8F1831CB5DFF8F407006800909E
:10846000DFF8F00700906946DFF8EC0701F018FC30
:10847000002801D000F05CFE0421002201AC2000A5
:1084800000F08AFEDFF8D407019001A9DFF8D007D9
:1084900001F080FD002801D000F04AFE13BD80B538
:1084A0000078002808D13B21DFF8B807008876DF84
:1084B000002801D000F03CFE01BD80B500F038FE80
:1084C00001BD18B587B01C2100226C46200000F0C9
:1084D00063FE002000905FF4A03001905FF4F02074
:1084E000029003208DF80C000020ADF80E00002053
:1084F0008DF81000DFF870070590DFF87007069020
:10850000684601F0BCFE002801D000F011FE08B062
:1085100010BD80B5002002F0F9F9002801D000F06C
:1085200007FE02F08FFA002801D000F001FE33DFD1
:10853000002801D000F0FCFD01BD80B5C0B20028CC
:1085400009D003280AD1022002F0E0F9002801D066
:1085500000F0EEFD02E0FFF7DCFFFFE701BD80B5B4
:108560000321DFF80C0702F081FC002801D000F0A5
:10857000DFFD01BD1CB50400208810280CD0112897
:1085800036D0132854D0212845D03B2868D0522813
:108590005AD056286CD073E0DFF8D816DFF8A8065A
:1085A000DFF8A826801AC008000450F0030001F08C
:1085B0007EF9072002F0AAF9002801D000F0B8FDEA
:1085C000A088DFF8A0160880DFF898060188DFF899
:1085D000880601F07BFB002801D000F0A9FDDFF840
:1085E000980600F00DFEDFF8900600F009FE47E067
:1085F000DFF88816DFF85006DFF85026801AC0082A
:10860000000450F0030001F052F94FF6FF70DFF85C
:108610005416088034E0DFF868060088ADF80000E2
:108620006946A0888FDF002801D000F081FD27E097
:10863000002300228521DFF82C0600887FDF002838
:1086400001D000F075FD1BE0002300220021DFF8BF
:1086500014060088B1DF002801D000F069FD0FE0AA
:108660001321A08876DF002801D000F061FD07E02B
:108670001321A08876DF002801D000F059FDFFE724
:1086800013BD80B502F082FD002801D000F050FD3E
:10869000002000906946012002F0F9FD002801D079
:1086A00000F046FD684602F0BEFE002801D000F052
:1086B0003FFD01BD10B5DFF8AC0500884A88904247
:1086C0001CD1088840F67722904217D18888C01EB6
:1086D000DFF8B0150880DFF8AC050388DFF8A405E3
:1086E0000288DFF8A415DFF86005DFF86045001B9D
:1086F000C008000450F0030001F0E6F810BD80B59A
:10870000DFF88815DFF8880503F07FF8002801D02E
:1087100000F00EFDF721DFF8780503F08FF8002850
:1087200001D000F005FD01BD0400FA0530B5A1B08F
:108730000178002905D0022900F05281C0F054814F
:1087400056E1DFF85005DFF850150978084400F0CD
:108750006EFEDFF844050078401CDFF83C15087019
:10876000DFF83005DFF830150978084410F8010CFF
:108770000A2813D0DFF81C05DFF81C150978084417
:1087800010F8010C0D2809D0DFF80C050078DFF88F
:10879000F414098880B28842C0F02181DFF8F8041F
:1087A00000780228C0F21881DFF8E8040078562823
:1087B00025D1DFF8E0044078652820D1DFF8D40423
:1087C000807872281BD1DFF8CC04C078492816D1F4
:1087D000DFF8C00400796E2811D1DFF8B8044079C1
:1087E00066280CD1DFF8AC0480796F2807D1DFF858
:1087F000AC040168DFF8A80400F002FDF8E0DFF83F
:1088000094040078512840F0B380DFF88804407861
:108810003D2840F0AD80DFF81404FEF78DFD002107
:108820000CE0DFF87024DFF870341B78CB181A44A2
:10883000DFF8F8335B5C02F8013C491C8142F0DB55
:10884000DFF8541409784018DFF84C140870DFF88A
:1088500048040078401CDFF8401408703B20DFF823
:108860003414DFF834241278114401F8020CDFF8D4
:10887000CC03FEF761FD00210EE0DFF81824DFF8DD
:1088800018341B78CB181A44DFF8A0330B4493F844
:10889000803002F8013C491C8142EEDBDFF8F8131E
:1088A00009784018DFF8F0130870DFF8EC0300785F
:1088B000401CDFF8E41308703B20DFF8D813DFF822
:1088C000D8231278114401F8020CDFF87403FEF784
:1088D00033FD00210EE0DFF8BC23DFF8BC331B784A
:1088E000CB181A44DFF844330B4493F8A03002F855
:1088F000013C491C8142EEDBDFF89C1309784018EB
:10890000DFF894130870DFF890030078401CDFF85C
:10891000881308703B20DFF87C13DFF87C23127883
:10892000114401F8020CC048FEF706FD00210DE0DD
:10893000DFF86023DFF860331B78CB181A44BB4B99
:108940000B4493F8403002F8013C491C8142EFDBB4
:10895000DFF8441309784018DFF83C1308700A2048
:10896000DFF83013DFF830231278114401F8010CDE
:1089700001A8802100F0ECFB00200020C549C64A78
:108980001278114401F8010CC248FEF7D5FC010031
:10899000802301AABF48FFF740FB05000A2001A978
:1089A00048556D1C012D17DB2800ADF80000AD48BF
:1089B00003886A4601A9AA4801F06CFB0400082C50
:1089C00008D0132C06D0052C04D02000002801D09C
:1089D00000F0AEFB132CE7D00020AF49087007E091
:1089E000406800F0A5FB03E0406800F0A1FBFFE752
:1089F00021B030BD80B58AB004A8AA491822FEF77C
:108A0000FDFCA94800904FF480700190A7480290A7
:108A10004FF4807003900723A54A694604A800F02C
:108A2000B3FC002801D000F083FB0BB000BD18B5EB
:108A3000ABB0AC2100226C46200000F0ADFB022060
:108A40008DF8000000208DF8020005208DF803004D
:108A50000120ADF84C009748149001208DF87C005F
:108A60004020229094482390944829906946804859
:108A700002F07BF9002801D000F05AFB01217C486C
:108A800002F070F92CB010BD0CED00E0600E030098
:108A90001C03030080B54FF48041002000F02CFD42
:108AA000002801D000F044FB02F054FF01BD80B566
:108AB00002F086FF002801D000F03AFB01BD80B52E
:108AC00000F017FF002801D102F087FF01BD80B53B
:108AD000FFF790FF1420FFF780FAFFF7DBFFFFF7A7
:108AE00021FBFFF7E4FF00F073F8FFF7CAFDFFF783
:108AF00021FBFFF704FEFFF7AEFCFFF798FFFFF73F
:108B0000E0FC6F4800F07CFB644801686D4800F0B1
:108B100077FB624801686B4800F072FB0A20FFF7A0
:108B20005CFA694800F06CFB4049684800F068FB5B
:108B30003D49674800F064FB4049664800F060FB2F
:108B4000654800F05DFB0A20FFF747FAFFF707FDD5
:108B5000FFF7B5FF384800780128F9D100203649E1
:108B6000087001F0C8FB72B600F011F8FFF724FAA4
:108B7000EEE70321594A1160594909680029FBD0E1
:108B800058490860564800680028FBD0704710B567
:108B90005548046855480068401E44432000FFF7CC
:108BA000E8FF0520FFF724FAC02220492000FEF745
:108BB00015FC4B4800680028FBD00020474908609E
:108BC000474800680028FBD00220FFF711FA10BDCB
:108BD00038B54548046845480068401E444320684D
:108BE00043490860206943490860206A4249086097
:108BF000206B424908604148006800903E48036885
:108C00003C4802683A4801683D4800F0F9FA3848A3
:108C1000006810F1010F05D0C022044D210028008A
:108C2000FEF7DCFB31BD0000602B0020202B002074
:108C3000580E03000C0B0300D7400020A02B00208F
:108C4000C02B0020E4040300B4FE02008CFE0200EE
:108C5000880F0300BF8102002C400020C781020062
:108C6000002B00209C2D00209F840200BB8402006A
:108C7000A02D0020700D0300200B0300300C03001A
:108C8000DA7302009E2D0020C0080300B5860200A2
:108C9000AC3F0020F8390020D8400020F42A002002
:108CA000DC080300A0090300F8370020F838002092
:108CB0002D8702001C2B0020401901003B8502007B
:108CC000F8080300400C030004060300340B030003
:108CD000500C0300600C03002806030004E501406B
:108CE00000E4014008E501401000001014000010ED
:108CF000AC400020B0400020B4400020B84000202C
:108D00004C06030080B5DFF8F80303F036F8DFF80F
:108D1000F413D1E90023002110185941DFF8E823AA
:108D2000D2E90023994206D801D3904203D2B0F190
:108D30007F4071F1FF3104BDD0E90223D1E9020186
:108D4000994204D301D8904201D3012000E00020D1
:108D5000C0B2704738B504000025DFF8B0030078D2
:108D6000012830D1002C2ED0207F00282BD0FFF7F7
:108D7000C9FFD4E9022399421FD301D890421CD3E2
:108D80002069002801D100202077A0696169884707
:108D90002069002817D0207F002814D0D4E90223AE
:108DA0002069002110185941C4E902012100DFF8AF
:108DB000600303F00BF8012505E02100DFF8500304
:108DC00003F004F801252800C0B232BD70B50500DB
:108DD0000E000D2400203070FFF794FFD5E9022328
:108DE000101A73EB01010122002399421ADB01DC06
:108DF000904217D3B0F5350F06D300F07BF902008F
:108E0000DFF81003821801E0D5E902235FF496032E
:108E10000021DFF8EC0202F013FF0400002C06D161
:108E200001200CE00021DFF8D80202F096FF0D2CA3
:108E300004D12800FFF78EFF3070FFE7002070BDDF
:108E400080B5DFF8CC0202F0D4FF002800D100206A
:108E500002BD80B5AE4840680068002800D10020FF
:108E600002BD80B5FFF7ECFF002801D0002101779B
:108E70000028F7D101BDA348D0E90001B0F17F403F
:108E800071F1FF319F4AC2E90001704780B5A248E5
:108E90000068002807D0A0480068FFF75BFF0020AB
:108EA0009D490860FFE701BD80B5FFF72BFF964A9B
:108EB000C2E9000101BD38B5050002E00020964975
:108EC0000860FFF7C6FF0024002836D092490968E1
:108ED000002901D1012415E0D0E902018E4A12686F
:108EE000D2E9022399420DD801D390420AD201243B
:108EF00089480068007F002804D0874801688448BA
:108F000002F064FFE4B2002C16D0FFF799FF0400D2
:108F100069462000FFF75AFF0028CFD07E4800683E
:108F2000002802D1280002F01DFE7B4804609DF855
:108F300000000028C5D107E006E077480068002857
:108F400002D1280002F014FE31BD80B56946734895
:108F5000006802F0FAFF0FE004E0FFF782FF012053
:108F60006A49087069466D48006802F0FDFF69466D
:108F70006A48006802F0E9FF002822D00178002941
:108F800003D00229E9D00CD3E6E74168097F002924
:108F900006D101214268117741685D4802F016FF51
:108FA000E0E741685C4A1268914203D100205A49C7
:108FB000086005E04168564802F028FFC0B200286A
:108FC000D0E701BD10B50400200002F0C0FE00286B
:108FD00001D0FFF750FF0021200002F0C6FE00285C
:108FE00002D02000FFF752FF0121200002F0BDFE59
:108FF000002802D02000FFF757FF2000FFF7A5FF51
:109000002000FFF758FF10BD80B53D4802F0BAFEC2
:1090100001BD38B504000D0069464048006802F003
:109020007AFF00280DD00470456069463B4800680F
:1090300002F080FF002802D0FFF7E6FFFFE70020E4
:1090400000E0042032BD1CB53548006800900823BC
:10905000582234493148006802F042FF002817D1F5
:10906000314A6946264802F03EFD0400002C01D03A
:1090700020000DE00121224802F062FE01232B4A6C
:1090800001211F4802F07AFD0120204908702000CC
:1090900016BD1300002B01D1072009E000684261D2
:1090A000C9B2012901D1012100E0002101610020A4
:1090B0007047D0B504000E00207F002801D00020AA
:1090C0000FE0A261FFF71EFE002780197941C4E975
:1090D00002012069002800D0266121000020FFF74E
:1090E00098FFD0BD80B50100002008770120FFF770
:1090F00090FF02BD80B5024802F03FFE02BD0000B5
:10910000D82A00204840002050400020D0400020B5
:10911000640D0300FFFFB40044400020700F030003
:10912000740F03007C3D0020C58F0200FFFF7F000D
:109130001FB5694600220023002481E81C0002902C
:109140006A46002144F2010002F02CFF1FBDFEE739
:10915000002202F055BFFEE70CB430B583B00446E0
:1091600006A802900A4600250194009502AB01A9C9
:10917000084878441E30FDF743F801990D70002827
:109180004EBF04460198041B204603B030BC5DF876
:109190000CFB00BFDBE1FFFF62F30F2262F31F4213
:1091A000401810F0030308D0C91A1FD3DB0748BFCB
:1091B00000F8012D28BF20F8022D130030B414460A
:1091C0001546103928BF20E93C00FAD8490728BFC6
:1091D00020E90C0048BF40F8042D890028BF20F882
:1091E000022D48BF00F8012D30BC7047C91818BFC8
:1091F00000F8012DCB0728BF00F8012D7047FEE7CE
:109200000EB4C0B5024603A800210190009101AB45
:109210000121044878440C30FCF7F2FF06BC5DF8ED
:1092200010FB00BF9D78000038B500239A4C0578EC
:10923000645D002C05D0D2B2001D03F07CF8030061
:1092400009E0954C0578645D002C04D1D2B20C3055
:1092500003F0CBFB0300180032BD80B500218E4A1D
:109260000378D25C002A04D0001D03F0BCF8010092
:1092700008E0894A0378D25C002A03D10C3003F05D
:10928000F5FB01000800C0B202BD38B50023824CD6
:109290000578645D002C05D0D2B2001D03F0B2F851
:1092A000030009E07C4C0578645D002C04D1D2B247
:1092B0000C3003F019FC0300180032BD010088686F
:1092C000C968081A7047E0B50178002947D002291B
:1092D00036D058D2017A002905D101226F49704851
:1092E000FFF7D3FF4FE0406801786E4803F0C6FDFA
:1092F000002808D001218DF80010019068466A49C5
:10930000096888470BE06748FFF7D8FF002806D0B8
:1093100000208DF800006846634909688847614865
:10932000FFF7CCFF5F498988814205D301225B4961
:109330005B48FFF7AAFF02E001205C49087022E0C9
:1093400002218DF80010C068019001225349544851
:10935000FFF79BFF684654490968884713E0544962
:10936000544803F09DFD002805D1012250494C4886
:10937000FFF75AFF06E003208DF8000068464A49CF
:1093800009688847FFE707BD70B588B005000C0085
:109390001E0045480260002C01D1072045E06268AC
:1093A00092B221683F4803F04DFD00283DD1E268AC
:1093B00092B2A1683F4803F045FD002835D16846C8
:1093C0003D492022FEF71AF868690690287C00289B
:1093D00001D1002000E001208DF814008DF81C6000
:1093E000687C002801D00E2000E000208DF81500D8
:1093F000E8680290A8680390286801906868009067
:109400002E4A6946264803F087FD00280DD100202A
:1094100026490870286810F1010F05D001221F4964
:109420001F48FFF732FF00E0002008B070BD38B5DC
:1094300001001E4804781B4803F032FD0500E4B229
:10944000002C0BD000201949087001221349144840
:10945000FFF71BFF002801D0FFF76AFE280032BD8E
:1094600010B50100C9B2134803F008FD0400002C38
:1094700010D10B48FFF7F1FE00280BD10C490D4825
:1094800003F00EFD002805D1012209490448FFF729
:10949000CBFE0400200010BDD9400020D2400020A7
:1094A000E02A0020E43F002094400020D340002028
:1094B000D1400020F43F00206C070300C792020057
:1094C00080B502681268904701BD80B5016849689F
:1094D000884701BD80B501688968884701BDC068BB
:1094E00001717047C068007970470121C0684171FF
:1094F0007047C0684079704780B5FF20DFF86C176F
:1095000088600020DFF8641708600020DFF85C172F
:1095100048600020DFF85417C1F818040020DFF875
:109520004C17C1F814040020DFF8401781F820041C
:10953000DFF83C0703F030FD00280AD1DFF83407DC
:1095400003F0F0FDDFF83017DFF83007081AC00825
:10955000002002BDDFF82007DFF82017401AC008FE
:10956000704710B50400C9B2002913D0FFF7F2FF0D
:10957000002100E0491C81420AD2DFF8042702EBF7
:109580008102128823689A42F4D12160002002E00F
:10959000052000E0002010BD01B5C9B26846FFF704
:1095A000E0FF002806D1DFF8DC06009900EBC100DF
:1095B000006800E0002002BDDFF8C82602EBC00012
:1095C000C9B2012906D00DD3032907D004D3042939
:1095D00006D007E0022006E0042004E0007902E063
:1095E000407900E00020C0B27047030000201A68F4
:1095F000C2F38002002A17D0187810F00300012867
:1096000002D0022808D00EE008681A68C2F383125C
:10961000921C1018086006E008681A68920D921CE7
:1096200010180860FFE70120C0B2704738B584B059
:109630000024DFF8540603F0DAFDDFF8500603F0EB
:10964000D6FDDFF8280640680090DFF82006856820
:10965000DFF818060099294000EB81000C3006E085
:10966000DFF808060099294000EB81000C306946BC
:10967000FFF7BBFF0028F3D100200DE0DFF8EC1569
:10968000009A2A4001EB8201C96801AA42F8201021
:109690000099491C0091401C0228EFD3019810F05A
:1096A000030001280BD0022812D1BDF80A4000980F
:1096B0000199890DC91C10EB9100009008E0BDF8DC
:1096C0000A4000990198C0F3831041180091FFE708
:1096D000DFF8B80503F090FD002803D00098DFF80C
:1096E0008C154860A4B2200005B030BD80B50021C3
:1096F000DFF89C0503F02AFD80F3100002BD2DE980
:10970000F84304000D0016001F00DDF82080A1467C
:109710005FEA1949FFF7EAFFDFF850157A1C18EAEB
:10972000020201EB820159EA0049C1F80C90DFF80E
:109730003C0518EA070700EB87000C30016864F36A
:10974000C5010160016866F389110160016865F374
:109750009F2101600121026861F30102026001683A
:1097600031F004010160BDE8F1832DE9FC41050001
:1097700088461400AE1C012700208DF800006846C2
:1097800003F094FDDFF8E4040068C8F80000DFF897
:10979000DC048068401CDFF8D4140968411ADFF843
:1097A000CC044068411817E00121DFF8E40403F01D
:1097B00003FDFFF73BFF0100DFF8D40403F0FCFCDE
:1097C000DFF8A8048068401CDFF8A0140968411A7B
:1097D000DFF8980440684118B142E5D33800C0B2C0
:1097E000002826D00021E4B2002C07D0012060F32D
:1097F000010151F0040165F3891106E0022060F3D4
:10980000010151F0040165F39F51DFF86024DFF896
:109810005C040368DFF854048068034002EB8300B3
:109820000C300160DFF8440400683618DFF83C04AF
:1098300006609DF8000003F03DFD3800C0B2BDE8B1
:10984000F6812DE9FC4104000D0017001E00DFF831
:109850001C04D0F80880012201A93000FFF785FF21
:10986000002818D00198801C00210AE0DFF8FC23B2
:1098700018EA000302EB830257F82130D360401C42
:10988000491CB142F2D3CDF80080019B320029007F
:109890002000FFF734FFDFF8D40390F820040028FD
:1098A00003D000F026F80028FBD1BDE8F38180B595
:1098B00000230022FFF7C5FF01BD80B50092012300
:1098C0006A46FFF7BEFF01BDE0B500920193022397
:1098D0006A46FFF7B6FF07BDDFF890034068DFF880
:1098E0008C130968884201D1012000E00020C0B239
:1098F00070472DE9F04385B0FFF7EEFF002801D057
:10990000002055E10020DFF86413C1F81804BFF30C
:109910004F8FDFF8580340680090DFF850038768E6
:10992000DFF848030099394000EB81000C30002437
:109930000025002106E0DFF834030099394000EBF0
:1099400081000C306946FFF750FE002813D0DFF885
:109950001C03D0F8180400280DD10098DFF80C1370
:1099600009688842E7D3DFF804030068DFF8FC12D7
:10997000486000201CE100200DE0DFF8F012009AA2
:109980003A4001EB8201C96802AA42F8201000990E
:10999000491C0091401C0228EFD3029810F00300EC
:1099A000022870D1DDF808805FEA98580298800D8F
:1099B000502804DADDF808905FEA995901E05FF079
:1099C0005009029869F39F50029019F1080102981A
:1099D000C0F3C200A64803F0E3FA0400002C00F034
:1099E0009480200003F02BFB2B00082202A920000A
:1099F00003F088FB08352E00781C00993940401A86
:109A0000800048452CD2002806D09849009A17407B
:109A100001EB87010C3100E09E49002801D00700CE
:109A200000E04F46002801D09A4D00E000250028B4
:109A300002D0B9EB000901E05FF0000933003A0001
:109A4000D2B2200003F05EFB56FA87F3002D13D04C
:109A50005FFA89F94A462900200003F053FB0BE026
:109A6000824800990F4000EB870010F10C01330091
:109A70004A46200003F046FB009818F1030810EB5B
:109A80009800009041E0029810F0030001283CD1BA
:109A90000298C0F38310062803DA0298C0F38310FB
:109AA00000E00620029960F3891102910298C0F348
:109AB0008311891C0298C0F3C20089006C4803F02E
:109AC0006FFA0400002C20D0200003F0B8FA2B001D
:109AD000082202A9200003F015FB083500260FE03C
:109AE0000098411C00912B0004226049384001EB92
:109AF000800010F10C01200003F004FB2D1D761CEA
:109B00000298C0F383108642EAD3002C33D0574822
:109B1000D0F810645548D0F81804002813D020005D
:109B200003F093FA3CE000253000FFF7E2FC012847
:109B300000D10125EDB2002D03D021003000FFF748
:109B4000BFFCF0680668002EEDD1200003F07DFA1E
:109B500000208DF8040001A803F0A8FB4348D0F8CA
:109B60001804002802D10098404948609DF804007C
:109B700003F0A0FB14E03D48D0F8104404E02000BE
:109B8000FFF7A8FCE0680468002CF8D1424943487C
:109B90003A4A801AC008000450F00200FFF787FE1E
:109BA000FFF79AFE002801D1012000E00020C0B29A
:109BB00005B0BDE8F08370B5002600E0761C0A2EE3
:109BC00013DA2A48D0F81044012501E0E06804685F
:109BD000002C05D02000FFF785FCB042F6D100250F
:109BE000EDB2002DEAD0300001E05FF0FF3070BD33
:109BF00038B50500FFF7DFFF040014F1010F01D1B4
:109C000020001EE020000100C9B22800FFF767FC19
:109C10001648D0F81004002806D11448C0F8105493
:109C20000020E96808600BE01048D0F81004C06814
:109C30000068E96808600D48D0F81004C068056045
:109C4000200032BD10B50948D0F810440120074962
:109C500081F8200407E02000FFF747FC2000FFF711
:109C600034FCE0680468002CF5D110BDD43100202C
:109C7000FC0B0300880D03000CFF02008CFE0200A9
:109C8000000000008CFE0200EC350020E8350020CA
:109C9000F0350020E0310020480B0300B4FE020044
:109CA000002801D10E2010E0002901D10E200CE087
:109CB0000278DE2A01D1082007E009684160DE2130
:109CC00001704FF6FF71418000207047002801D1DC
:109CD0000E2006E00278DE2A01D0082001E0418053
:109CE0000020704780B50200107A00280ED00021B5
:109CF000508866DF002802D10020107206E011288B
:109D000002D10120107201E05168884701BD80B581
:109D10000A79012A07D109884288914203D1012199
:109D20000172FFF7DFFF01BD70477FB504000D0032
:109D300028886188884224D1AE1C3078022820D13E
:109D4000307A042805D0307A062802D0307A0528E7
:109D500017D168461021FFF7FBF902208DF80000AB
:109D60004FF4C070ADF80400307A052802D100200D
:109D7000ADF8040069462888B0DF002801D061688A
:109D800088477FBD38B505000C00002C2CD0002D75
:109D90002AD02078DE2827D1A8886188884202D17D
:109DA0002000FFF79FFF2888012806D0022809D04D
:109DB000112811D051280AD016E0291D2000FFF7E4
:109DC000A6FF11E0291D2000FFF7AEFF0CE0291DC2
:109DD0002000FFF7AAFF07E0A8886188884202D127
:109DE0004FF6FF706080FFE731BDFEE770B58AB0C7
:109DF00004000D00002000906A46A988606903F005
:109E00005EFA00280821002202AE3000FFF7C4F9F4
:109E100001A803900220ADF808000020ADF80A0068
:109E200002AA2189A888ADDF00281FD1A0690028D7
:109E30001CD0039803F07FFA002817D00098002860
:109E400002D00120009908701821002204AE3000D1
:109E5000FFF7A2F902208DF810000594A888ADF84C
:109E600018000098079004A8A16988470AB070BD3F
:109E7000F0B587B004000E00B51D6A46B188606970
:109E800003F01DFA00281821002201AF3800FFF767
:109E900083F90294B088ADF80C00009804902888EB
:109EA000218988421FD1688902281CD10098002886
:109EB0002CD015F10C0003F03EFA002806D001204A
:109EC0000099087002208DF8040005E00020009938
:109ED000087003208DF80400A069002816D001A89E
:109EE000A169884712E02888A18988420ED1A0691B
:109EF00000280BD000208DF8040015F10C0005900F
:109F00006889ADF8180001A8A169884707B0F0BDBD
:109F100078B587B004000D006A46A988606903F02F
:109F2000CEF9002815D100980078002811D018210A
:109F3000002201AE3000FFF72FF901208DF8040058
:109F40000294A888ADF80C000098049001A8A169BB
:109F5000884708B070BD80B50A00002A01D00028EB
:109F600000D116E00188102904D0502907D05729C4
:109F70000AD00EE001001000FFF738FF09E00100F1
:109F80001000FFF775FF04E001001000FFF7C0FFAD
:109F9000FFE701BD30B58DB004000D0009A83C49B4
:109FA0001022FDF72BFA002C01D10E206EE0002DBF
:109FB00001D10E206AE02868A061210009A862DFB3
:109FC000002863D120788DF802000120ADF8000050
:109FD000A21C69460120A8DF002857D120210022B9
:109FE00001AD2800FFF7D8F80220ADF80400207872
:109FF0008DF80600F420ADF808000120ADF80A0045
:10A0000001208DF810009DF8110050F008008DF827
:10A0100011009DF8110050F004008DF8110001208E
:10A020008DF8150001208DF8160014F10C0201A91D
:10A03000608803F0E4F9002828D12021002201AD36
:10A040002800FFF7A9F80320ADF8040020788DF868
:10A050000600F420ADF808000120ADF80A00012048
:10A060008DF810009DF8110050F010008DF81100CF
:10A0700001208DF8150001208DF8160001208DF8C3
:10A080001700221D01A9608803F0B9F90DB030BD99
:10A09000200C03002DE9F84185B004000D001600E6
:10A0A0001F00002C01D10E2030E06A46390089B231
:10A0B000606903F004F9002828D1380080B24FF617
:10A0C000FF71884202D00098002801D105201DE0D0
:10A0D00000980078002801D1082017E03088F52882
:10A0E00001DB072012E0102100220DF10408404698
:10A0F000FFF752F8A088ADF80400049503960120FC
:10A100008DF8060001A9380080B2AEDF06B0BDE8C8
:10A11000F081FEE7002100E0491C002910D1DFF8A2
:10A120008C23142303FB01F3D25A03009BB29A42FF
:10A13000F2D1DFF878231420414302EB010000E064
:10A140000020704780B50180002101720A30DFF8DD
:10A1500060130822FDF742F901BD4FF6FF7101803F
:10A160007047F0B4848814FA82F415008688ADB282
:10A17000B54201D292B200E082888588AA1AC588C9
:10A1800015FA83F51E00C788B6B2BE4201D29BB253
:10A1900000E0C388C688F31A4E880788BE4203D3FE
:10A1A00040884E88B04201D2002010E0888890425A
:10A1B00002D38888844201D2002008E0C8889842EF
:10A1C00002D3C888854201D2002000E00120F0BC03
:10A1D000704780B5DFF8DC128969002903D0DFF809
:10A1E000D4128969884701BD10B580B275DF0400BB
:10A1F000002C04D0112C02D02000FFF7EAFF002C25
:10A2000001D1012000E00020C0B210BD38B505002A
:10A21000280080B2FFF77EFF0400002C2ED0207AA9
:10A22000A449097B88420CD214F10A01280080B2AB
:10A23000FFF7DAFFC0B2002820D0207A401C20723D
:10A240001CE0002020729B48007C002809D03B21A4
:10A25000280080B276DF002803D0082801D0FFF75D
:10A26000B8FF94484069002808D000208DF800000D
:10A27000ADF8025068468F494969884731BD38B505
:10A280000400002C01D10E2034E08A4821001C2259
:10A29000FDF7B4F8864887490860206800280AD08E
:10A2A00020687ADF002825D1814821680822FDF73F
:10A2B00095F8002405E07E487BDF0028F9D019E0FE
:10A2C000641C002C15D17948142101FB04F100EB2A
:10A2D00001052800FFF741FF7748610108446860E5
:10A2E000764A0021281DFEF7D4FE0028E8D003207E
:10A2F00000E0002032BD10B5002401E0FFE7641C3F
:10A30000002C12D16948142101FB04F10844406873
:10A31000FEF7E8FE0028F1D0042802D00828EED08D
:10A3200001E0112002E0032000E0002010BD80B514
:10A3300002000B00587A002810D1187A002802D1A8
:10A340005C48416801E05B48816892B25868FEF75A
:10A35000B0FE002811D0FFF73CFF0EE0002018727D
:10A3600054484069002808D001208DF80000ADF85D
:10A37000022068464F494969884701BD70B505000C
:10A38000E87BAE88C0B2012823D14FF6FF70FFF7FB
:10A39000C1FE0400002C03D10420FFF71AFF18E0CF
:10A3A000310089B22000FFF7CDFE4FF6FF7340F277
:10A3B000F31215F1100114F10A00FFF7D2FE6072DA
:10A3C0003C48C089002804D12100300080B2FFF74A
:10A3D000AEFF70BD10B5808880B2FFF79BFE040011
:10A3E000002C09D06068FEF77DFE002801D0FFF741
:10A3F000F0FE2000FFF7B1FE10BD70B5851D298865
:10A400002C4AD28991421DD1698902291AD18688A4
:10A41000300080B2FFF77EFE0400002C12D015F150
:10A420000C0002F088FF002805D02100300080B227
:10A43000FFF77DFF06E06068FEF754FE002801D0BC
:10A44000FFF7C7FE70BD70B50500AE88300080B262
:10A45000FFF760FE0400002C0FD04FF6FF7340F2B0
:10A46000F31215F1080114F10A00FFF77AFE607289
:10A470002100300080B2FFF75AFF70BD80B501881F
:10A48000102906D0112907D012290BD0502906D047
:10A490000BE0FFF773FF08E0FFF79CFF05E0FFF715
:10A4A000ACFF02E0FFF7CFFFFFE701BD983F0020C0
:10A4B00058400020043F0020203F00200DA2020051
:10A4C0005FF0A040704711B581B00C0001A8FFF704
:10A4D000F7FF019900EB8101D1F8001731F4403109
:10A4E000019A00EB8202C2F80017019900EB81018A
:10A4F000D1F80017E4B251EA0441019A00EB82005E
:10A50000C0F8001713BD10B5DFF8780400780028F4
:10A5100009D00024042C08D2022C02D0200003F021
:10A52000C7F8641CF6E703F0CAF810BD38B505009B
:10A5300000240020DFF850040078002805D0002017
:10A54000DFF844140870FFF7DEFF2800C0B20028CF
:10A5500037D0022841D040D3042800F0B28076D30F
:10A56000062800F02081C0F0E780082800F02F8145
:10A57000C0F027810A2800F04881C0F037810C28FC
:10A5800000F06181C0F050810E2800F06181C0F0C0
:10A590005F81102800F05C81C0F05A81122800F021
:10A5A0008E81C0F05581142800F09681C0F08C8116
:10A5B000162800F0A481C0F09781172800F09F8131
:10A5C000A2E1FFF7A0FFDFF8C4030068FEF78AFDF1
:10A5D0000400DFF8BC03057096E1002003F053F897
:10A5E00000280CD0002003F063F82800C0B2022835
:10A5F00002D14FF4E1600DE04FF47A600AE00020F0
:10A6000003F04FF82800C0B2022801D1C82001E0B1
:10A610004FF4C870DFF878130D70002214004FF467
:10A620000041A1FB000110F57A7051F100014FF4D7
:10A63000FA620023FCF726FF02000B001100220043
:10A64000DFF848030068FEF734FD04005CE10020F9
:10A6500003F019F800280CD0002003F029F8280096
:10A66000C0B2032802D14FF448700DE04FF47A6075
:10A670000AE0002003F015F82800C0B2032801D139
:10A68000C82001E04FF4C870DFF804130D700022F9
:10A6900014004FF40041A1FB000110F57A7051F154
:10A6A00000014FF4FA620023FCF7ECFE02000B00FD
:10A6B00011002200DFF8D4020068FEF7FAFC040063
:10A6C00022E1002002F0DFFF00280CD0002002F081
:10A6D000EFFF2800C0B2042802D14FF47A600EE0E8
:10A6E0004FF47A600BE0002002F0DBFF2800C0B2DC
:10A6F000042802D14FF4C87001E04FF4C870DFF8AD
:10A7000090120D70002214004FF40041A1FB0001D3
:10A7100010F57A7051F100014FF4FA620023FCF752
:10A72000B1FE02000B0011002200DFF86002006899
:10A73000FEF7BFFC0400E7E0002002F0A4FF0028C1
:10A740000BD0002002F0B4FF2800C0B2052801D1D0
:10A75000C8200DE04FF47A600AE0002002F0A1FF6B
:10A760002800C0B2052801D1C82001E04FF4C8700C
:10A7700087490D70002214004FF40041A1FB000135
:10A7800010F57A7051F100014FF4FA620023FCF7E2
:10A7900079FE02000B00110022007C480068FEF7E1
:10A7A00088FC0400B0E0002002F09DFF78480570AE
:10A7B000002240F2666175480068FEF77AFC0400EA
:10A7C000A2E0002002F06DFF714805709CE00120BE
:10A7D0006D490870012002F086FF002240F2666198
:10A7E0006A480068FEF765FC04008DE001206649B8
:10A7F0000870012002F077FF00224FF400516348F7
:10A800000068FEF756FC04007EE001205E490870F7
:10A81000012002F068FF002240F266615B48006898
:10A82000FEF747FC04006FE0012057490870012043
:10A8300002F059FF00224FF4005154480068FEF71F
:10A8400038FC040060E002F044FF514805705BE012
:10A8500050480068FEF746FC0400EDB2D5F1110542
:10A86000002D25D0002C23D1022D1AD30022140054
:10A87000ADB2C82045434FF4004080FB050110F500
:10A880007A7051F100014FF4FA620023FCF7FAFDEF
:10A8900002000B00110022003E480068FEF709FC90
:10A8A0000400022002F0FDFE01203649087005E098
:10A8B000022002F0FDFE00203249087024E0FFF77C
:10A8C00022FE334805701FE0FFF71DFE002002F056
:10A8D000E8FE2F48057017E0FFF715FE012002F093
:10A8E000E0FE2B4805700FE0FFF70DFE002002F0A0
:10A8F000D8FE012002F0D5FE2548057004E002F0E4
:10A90000E8FE23480570FFE7200032BD80B5002136
:10A91000214A1278D20703D5C0B2FFF707FE010023
:10A92000080002BD10B40023042824D21400E4B2AD
:10A93000012C07D10A00D2B2012A02D110F10E0275
:10A9400000E00022C9B200290DD0022905D010D2A2
:10A950000B4C0321484322540EE0094C0321484389
:10A960002044427008E0064C032148432044827092
:10A9700002E0072300E00723180010BC7047000026
:10A9800020400020D6400020D5400020800F03004A
:10A99000D4400020840F03009840002010B5042804
:10A9A0000DD2C9B2002901D0032400E0002402F036
:10A9B000A0FE2100C9B2FFF786FD002000E00620BE
:10A9C00010BD80B50121FFF7E9FF02BD80B501226E
:10A9D00000210020FFF7A6FF002801D0072812D190
:10A9E000072202210120FFF79DFF002801D0072840
:10A9F00009D1042202210020FFF794FF002801D092
:10AA0000072800D1002002BD80B5012202210020CC
:10AA1000FFF788FF002801D0072812D10722022162
:10AA20000120FFF77FFF002801D0072809D10A2263
:10AA300000210020FFF776FF002801D0072800D171
:10AA4000002002BD80B50020FFF7BBFF002801D029
:10AA5000062807D10120FFF7B4FF002801D00628FF
:10AA600000D1002002BD80B50088102802D0112836
:10AA700015D029E01548006800280AD1FFF7A6FF85
:10AA8000002806D012490968002902D01049096837
:10AA900088470E480068401C0C49086014E00B48C9
:10AAA0000068401E094908600848006800280AD16B
:10AAB000FFF7AAFF002806D005490968002902D03F
:10AAC000034909688847FFE701BD0000A040002056
:10AAD0009C40002090F830047047002200E0521C97
:10AAE000062A04D2815C0029F9D0012000E0002070
:10AAF0007047C0B2401C052190FBF1F201FB12002F
:10AB0000C0B27047CA7B012A02D18988A0F82414F8
:10AB1000704710B50400002084F82E048888B4F82B
:10AB2000241488420DD1207900280AD10121200067
:10AB300000F09CF9002804D0A16B002901D0A16B82
:10AB4000884710BD10B504000888262814D1087A5B
:10AB5000012802D0087A02280ED1A078FFF7C9FF99
:10AB60000100C9B2200000F081F9002804D0A16BD7
:10AB7000002901D0A16B884710BD38B504000D0035
:10AB800004F22740FFF7A9FFEDB2012D06D024D330
:10AB9000032D18D00FD3042D1AD01EE0A17900295F
:10ABA00009D094F82410002905D10100C9B2002968
:10ABB00001D0012012E0E179002904D0C0B20028C0
:10ABC00001D002200AE0207A002801D0032005E00D
:10ABD000607A002801D0042000E0002032BD01226C
:10ABE00080F831200022C0F8202400F2264048607E
:10ABF0000020886002200870802088810020704733
:10AC0000022280F8312090F82420002A02D0072266
:10AC10000A7001E003220A7002698A810022C0F8EA
:10AC2000202400F226424A60C068886000207047F5
:10AC300080B54179002909D090F82E14002905D15A
:10AC4000FFF748FF002801D0012000E00020C0B23B
:10AC500002BD38B504000D000122B4F81414D4F874
:10AC6000100403F0BFF8002800D0057014F13C0276
:10AC700014F5826114F1540072DF32BD38B504005E
:10AC80000D006069A860A069A88194F824000028DC
:10AC900003D0062084F83C0002E0012084F83C0048
:10ACA0002000FFF7C5FF00280BD0022028750421E3
:10ACB0002000FFF7CEFF00280BD1052084F83100DB
:10ACC00002E0032084F8310014F58260C4F8200407
:10ACD000002032BD38B504000D00E069A860206A8C
:10ACE000A88194F82400002803D0062084F83C00B2
:10ACF00002E0012084F83C002000FFF799FF0028C3
:10AD00000BD00220287504212000FFF7A2FF0028A5
:10AD10000BD1062084F8310002E0042084F83100D1
:10AD200014F58260C4F82004002032BD8178012926
:10AD300005D190F82010012901D1002008E0816A96
:10AD4000042902D0406A042801D1002000E001203B
:10AD5000704790F82400012801D1EE2000E01F2068
:10AD600080B2704780F83010704770B504000D0055
:10AD7000002D01D0002C01D10E206CE015F17800DF
:10AD8000FFF7D4FF002801D1072064E00020A07065
:10AD9000201D15F178012C22FCF730FB002084F8EF
:10ADA0003000D5F8A4006063D5F8A800A0634FF682
:10ADB000FF70A4F8240414F58260C4F8200407216D
:10ADC000002204F226463000FEF7E6F9207800283B
:10ADD00002D1FF2084F8540014F15500C4F8100487
:10ADE0002000FFF7B6FFA4F8140404F2144214F193
:10ADF0005501280002F01EFF00282CD104F231205A
:10AE0000C4F818042000FFF7A4FFA4F81C0404F2FF
:10AE10001C42D4F8181415F13C0002F00BFF002876
:10AE200019D1012084F85100A069A4F8480001203C
:10AE300084F83C0000202064002084F85000606901
:10AE4000606414F13C02002114F1540072DF002808
:10AE500001D10121217070BD0168012902D0006873
:10AE6000022801D1012000E00020704770B50400E5
:10AE70000D002078002801D10820B5E0A570072139
:10AE8000002204F226463000FEF786F9A079002859
:10AE900002D0A07801280BD0E079002802D0A07859
:10AEA000012805D0E07900280FD0A07802280CD125
:10AEB000606B002806D0012084F82D040820616B07
:10AEC000884702E0002084F82D042900C9B2200040
:10AED000FFF753FEA070606B002816D0A0780328FF
:10AEE00002D0A078042810D1607900280DD094F801
:10AEF0002E04002809D1002084F83004012084F8B1
:10AF00002F040720616B884702E0002084F82F049B
:10AF10001821002214F13C052800FEF73DF901201C
:10AF200084F83C0014F12C00FFF796FF002803D0B2
:10AF3000E06A84F8510002E0012084F8510094F89E
:10AF4000240000280CD014F12800FFF785FF00280A
:10AF500003D0A06A84F8520002E0012084F8520075
:10AF6000002084F85000A07800281ED002280AD0C3
:10AF700003D3042813D00CD31BE014F13C012000B0
:10AF8000FFF72DFE15E014F13C012000FFF738FE1D
:10AF90000FE014F13C012000FFF770FE09E014F10E
:10AFA0003C012000FFF796FE03E0002084F831000A
:10AFB000FFE7A07800280FD014F13C02D4F8201449
:10AFC00014F1540072DF00280ED194F8301094F878
:10AFD000540073DF002807D1606B002803D094F879
:10AFE0003100616B8847002070BD80B50A00018880
:10AFF000102904D0112907D026290AD00EE001001B
:10B000001000FFF77FFD09E001001000FFF781FD50
:10B0100004E001001000FFF795FDFFE701BDFEE72A
:10B02000012210F01F018A40DFF8101240B24009DF
:10B0300041F820207047010049B2002909D5DFF806
:10B04000001240B210F00F00084410F8040C400940
:10B0500004E0DFF8F01140B2085C400970478068F6
:10B0600070470100080040B2202805DADFF8D80157
:10B07000C84010F001000EE0080040B2402809DA94
:10B08000012020398840002801D0012000E0002064
:10B09000C0B200E001207047082803D2EC21014132
:10B0A000C80701D4002000E00120704710B504005B
:10B0B000200040B2FFF7D5FF002802D142F2010084
:10B0C00024E0200040B2FFF7B6FFFFF7E5FF0028BD
:10B0D00002D142F2020019E05C488068002810D0DA
:10B0E0005A48210049B2490950F82110012214F0B0
:10B0F0001F0082401143554864B2640940F824108F
:10B1000003E0200040B2FFF78BFF002010BD1FB509
:10B1100004004F49684602F090FE02E0684602F0E3
:10B1200093FE6846FFF79BFF00280BD06846FFF7A9
:10B1300096FF026841682000C0B290470028EDD118
:10B14000112000E0002004B010BD1FB504004149EB
:10B15000684602F072FE0AE06846FFF780FF026868
:10B1600041682000C0B29047684602F06DFE684614
:10B17000FFF775FF0028EFD11FBD80B51620FFF740
:10B1800095FF002801D0FDF7D3FF01BD1CB5324863
:10B190000078002801D0082036E001202F490870EF
:10B1A0000020FFF7B4FF112801D100202CE000207F
:10B1B000FFF7CBFF2A480068019000208DF80000BF
:10B1C000684602F073F8274901A810DF0400002C3C
:10B1D00003D101202049087002E000201E490870B8
:10B1E0009DF8000002F066F8002C01D020000BE072
:10B1F00000201A49087000201B490870FFF7BDFFA6
:10B200000120FFF7A2FF002016BD13480078704709
:10B21000E0B51649684602F010FE08E06846FFF700
:10B220001EFF016840688847684602F00DFE6846C8
:10B23000FFF715FF0028F1D107BD000000E100E095
:10B2400018ED00E000E400E0FC06FFBD1440002023
:10B25000B80D0300C40D0300DC400020DE400020D8
:10B26000940F0300A5BF0200DD400020D00D0300B5
:10B2700080B5FFF7CDFF01BD80687047002801D180
:10B280000E2003E0A24909680160002070477FB5E5
:10B2900005000C002000FFF7F1FF002840F0B98006
:10B2A0000C2100226E463000FDF776FF8DF800502D
:10B2B00001208DF802000620ADF8040022686946DE
:10B2C000202069DF00280CD002F0D2FD0200914955
:10B2D0009148924BC01AC008000450F00100FEF7DC
:10B2E000ECFA0C2100226E463000FDF755FF0120DC
:10B2F0008DF8010000208DF8020000208DF8030079
:10B3000022686946402069DF00280CD002F0B0FDB9
:10B31000020083498048814BC01AC008000450F0E5
:10B320000100FEF7CAFA0C2100226E463000FDF73C
:10B3300033FF8DF80050F720ADF80200226869460F
:10B34000232069DF00280CD002F092FD020075492D
:10B350007148724BC01AC008000450F00100FEF79B
:10B36000ACFA0C2100226D462800FDF715FF0120E4
:10B370008DF8000022686946012069DF00280CD0A2
:10B3800002F076FD020068496348644BC01AC008A9
:10B39000000450F00100FEF790FA0C2100226D46E7
:10B3A0002800FDF7F9FE4FF4B0600090226869466E
:10B3B000A12069DF00280CD002F05AFD02005B4991
:10B3C0005548564BC01AC008000450F00100FEF763
:10B3D00074FA0C2100226D462800FDF7DDFE9DF871
:10B3E000000010F0FE008DF8000022686946A020E1
:10B3F00069DF00280CD002F03BFD02004C494648B2
:10B40000464BC01AC008000450F00100FEF755FA80
:10B41000002004B070BD474800684FF48061484385
:10B4200010F10050704770B506003568300060DFDD
:10B4300004003068854225D23F493748374A801A90
:10B44000C008000450F00200FEF731FA33682A0009
:10B450003A493148314D401BC008000450F0020009
:10B46000FEF732FAFFF7D7FF02003068121A3449AC
:10B4700029482A4BC01AC008000450F00200FEF709
:10B480001CFA01E03068A842002C03D101202D49AC
:10B4900008700DE0200002F0EBFC02002A491E4873
:10B4A0001E4BC01AC008000450F00100FEF705FA58
:10B4B000200070BD18B5ADF5017D22480078002848
:10B4C00016D103E0052801D0FDF732FE0DF5027D0F
:10B4D00010BD01A8FFF7D0FE026841682000904728
:10B4E00001A802F0B1FC01A8FFF7C6FE0028F0D1C8
:10B4F0004FF4FA70ADF80000694604A861DF002837
:10B50000E0D104AC114901A802F097FCEBE7000080
:10B51000980F030044020300CCFE02008CFE0200E0
:10B52000AC0103008C020300F80103006400030077
:10B53000B80003000C010010B40403005004030021
:10B5400010050300DF4000208C070300E80D030016
:10B55000F7210180172141800021017100214171F3
:10B56000FB2181711B21C171704738B584B0050082
:10B57000DFF8A803D0E90023CDE90223ADF80810D5
:10B58000ADF80A10DFF89803D0E90023CDE90023D5
:10B590006A4602A9280080B290DF0400002C3ED049
:10B5A000200002F065FC0300ADB22A00DFF874133E
:10B5B000DFF87403DFF87453401BC008000450F038
:10B5C0000100FEF781F9BDF80000002803D1BDF8A5
:10B5D0000200002810D0BDF80230BDF80020DFF8CE
:10B5E0005013DFF84403DFF84453401BC008000445
:10B5F00050F00100FEF768F9BDF8040000280ED0F5
:10B60000BDF80420DFF82C13DFF81C03DFF81C332F
:10B61000C01AC008000450F00100FEF74EF92000E7
:10B6200005B030BD38B58C88220092B200EBC20262
:10B63000951D0279AA71C97B012902D0022903D084
:10B6400005E00088288002E040882880FFE76888BD
:10B65000298888421DD22988200080B2A5DF0028D1
:10B6600002D10120687114E0112802D10120287153
:10B670000FE002F0FDFB0200DFF8BC12DFF8A802C9
:10B68000DFF8A832C01AC008000450F00100FEF72D
:10B6900014F9E879A979884205D2A97989B22000FC
:10B6A00080B2FFF762FF31BD80B5898800EBC10031
:10B6B000801DFFF74DFF01BDFEB58A884989130043
:10B6C0009BB200EBC3039C1D0B0025889BB2AB42D1
:10B6D00000D3218861806188172901DA172100E0F1
:10B6E00061886180016900290FD0617900290CD03F
:10B6F0009249D1E90067CDE90067ADF80220618881
:10B70000ADF804106946026990470020607100207E
:10B710002071F7BD7CB504008D88C888290089B2E6
:10B7200004EBC1018E1D010089B2172901DA17202F
:10B73000FFE70100328889B2914200D330887080DF
:10B74000002030713188280080B2B5DF00280CD08D
:10B7500002F08EFB02007A497348744BC01AC0088D
:10B76000000450F00100FEF7A8F87079002810D10D
:10B77000206900280DD07348D0E90023CDE90023CB
:10B78000ADF802507088ADF80400694620002269C7
:10B79000904773BD18B58DB0040002A8091D2C2276
:10B7A000FBF72CFEBDF80810BDF80C000A0092B2A1
:10B7B00004EBC20250732069002810D06248D0E91F
:10B7C0000023CDE90023ADF8021089B204EBC100DB
:10B7D000407B8DF8040069462000226990470EB036
:10B7E00010BD10B50A1D118800EBC100801D9188A5
:10B7F00083790C00E4B2A34201D28179FFE7C9B298
:10B8000089B21088FFF7B1FE10BD38B50500002DD4
:10B8100001D10E2011E02961F7202880F7206880EF
:10B82000FB202871002405E005EBC400801DFFF714
:10B830008FFE641C002CF7D0002032BD002801D1FF
:10B840000E2008E00A0092B2173AE12A01D307203D
:10B8500001E001800020704738B50D008488210088
:10B8600089B2002957D1018810290AD011290DD099
:10B8700023291FD0242918D03A290CD055290FD0BC
:10B880001DE001002800FFF7CDFE18E001002800B0
:10B89000FFF70AFF13E001002800FFF70DFF0EE09D
:10B8A00001002800FFF736FF09E001002800FFF73C
:10B8B00071FF04E001002800FFF793FFFFE720007D
:10B8C00080B205EBC000807A002824D0200080B22E
:10B8D00005EBC000C188200080B2A5DF00280BD195
:10B8E0000020210089B205EBC10188720120A4B2B9
:10B8F00005EBC401C8720EE011280CD002F0B8FAB2
:10B9000002000D490848094BC01AC008000450F055
:10B910000100FDF7D2FF31BD00000000700E0300F2
:10B92000680E030060010300A4FE02008CFE02000A
:10B93000600303000C0003001C040300780E0300E6
:10B9400084040300800E0300880E03000121C068F8
:10B950004171704780B55FF0FF3002F0C9FA0421F1
:10B960000348FEF745F90248FFF7F0FF01BD00006C
:10B97000100D0300012210F01F018A401D4940B242
:10B98000400941F82020704700210160BFF35F8F1C
:10B99000704780B500208DF80000684601F086FCF5
:10B9A000F1EE100A30F09F00E1EE100ABFF35F8F56
:10B9B0002620FFF7DFFF9DF8000001F07BFC01BDB2
:10B9C00080B500200C4908700C48FFF7DDFF0C49DA
:10B9D0000C4802F032FA002002BD80B5FFF7D9FF13
:10B9E000FFF713FC002801D041DF02E020BF40BF79
:10B9F00020BF01BD80E200E0DB400020C440002009
:10BA0000AC0D030038400020012210F01F018A40D5
:10BA1000DFF88C1340B2400941F820207047012222
:10BA200010F01F018A40DFF87C1340B2400941F852
:10BA300020207047020052B2002A09D54901DFF8E0
:10BA4000682340B210F00F00104400F8041C04E01A
:10BA50004901DFF8582340B21154704780B5C9B28C
:10BA600040B2FFF7E7FF01BD80B540B2FFF7CCFF62
:10BA700001BD80B5002806D0DFF8342352F0010262
:10BA800040214843904701BD00EB8100C0F84025AC
:10BA9000704700EB8100D0F840057047C0F80413F0
:10BAA0007047C0F80813704709B24058704781B01A
:10BAB00000220B001BB2C25009B2405800900098FF
:10BAC00001B07047D0F804057047C0F808157047FA
:10BAD000012250FA81F002607047C0F844137047A9
:10BAE000C0F84813704738B504000D00B1486179BB
:10BAF00040F82120B048617900EBC10000790028AE
:10BB00000CD00824AD49AE48AE4A801AC0080004E3
:10BB100050F00200FDF7CBFE200022E029882068CB
:10BB2000FFF7D3FFA97894F90400FFF797FF94F982
:10BB30000400FFF799FFA048617900EBC1000121E3
:10BB400001719D48617940F8314000249E499C482C
:10BB50009C4A801AC008000450F00300FDF7A7FEBD
:10BB6000200032BD80B500210068FFF7B1FF01BDA4
:10BB700080B504210068FFF7ABFF01BD2DE9F84354
:10BB800005000E0017001C005FF4803818FA06F854
:10BB90005FEA860919F5A07927F07F4741462868B2
:10BBA000FFF77FFF41462868FFF79AFF494609B231
:10BBB0002868FFF77CFF3A0031002868FFF764FF30
:10BBC00041462868FFF789FFE4B2002C03D04146C4
:10BBD0002868FFF763FFBDE8F18370B505000E002C
:10BBE000140031002868FFF778FFE4B2002C03D07E
:10BBF00031002868FFF752FF70BD38B504000D0012
:10BC000029002068FFF76CFF29002068FFF749FF33
:10BC100031BD38B504000D00290009B22068FFF7D6
:10BC200043FF002806D0290009B22068FFF73FFF34
:10BC3000012000E0002032BD401A20F07F40704714
:10BC40002DE9F84F06000F001D005FF4803818FA48
:10BC500007F85FEA870919F5A07922F07F421400FE
:10BC600041463000FFF7C9FF3068FFF72BFF8246DF
:10BC700039003068FFF70DFF8346524639003068BF
:10BC8000FFF702FF494609B23068FFF710FF51463F
:10BC90005846FFF7D1FF012807D11020FFF7E9FE32
:10BCA000494609B23068FFF702FF3068FFF70AFF24
:10BCB000814649462000FFF7BFFF82464146306873
:10BCC000FFF70BFFBAF1010F0FD1641C22003900FE
:10BCD0003068FFF7D9FE1020FFF7CBFE3068FFF782
:10BCE000F1FE814524D00D2028E022003900306883
:10BCF000FFF7CAFE3068FFF7E5FE81464946601E41
:10BD0000FFF79AFF7FF07F414D1B854201D20D2046
:10BD100014E000280CD1641C220039003068FFF7C1
:10BD2000B3FE3068FFF7CEFE814501D00D2005E05F
:10BD3000012241463000FFF750FF0020BDE8F28F9E
:10BD400080B50A00D2B20221FFF747FF01BD80B5DE
:10BD50004FF48271FFF75DFF02BD80B55FF4803262
:10BD600012FA01F1FFF749FF01BD80B5890011F515
:10BD7000A07109B2FFF74DFF02BD80B50068FFF763
:10BD8000A1FE02BD80B590F90400FFF748FE01BD99
:10BD900080B50948006807490968884701BD000067
:10BDA00000E100E000E200E018ED00E000E400E067
:10BDB000500E0300A440002060400020E005030076
:10BDC00094FE02008CFE0200E40A030070B5040039
:10BDD0000D00666800E036683068002805D029004C
:10BDE0003068A26890470028F5D130682860356037
:10BDF00070BD02005068006851680968002904D0CD
:10BE00005168096809685268116070470200002093
:10BE1000536800E01B681A68002A05D01A688A4235
:10BE2000F8D1086818600120C0B270471CB450E80F
:10BE3000014FA2B2C3891A4483899A4228BFD21AF9
:10BE400003899A4202BFBFF32F8F002007E0C2EAA6
:10BE5000040240E80123002BE9D14FF001000194D6
:10BE60008DF80000019808609DF8000016BC70472E
:10BE700050E8012FC2EA024240E801210029F7D12F
:10BE8000704700001CB450E8024F1FFAA4F2C388A8
:10BE90009A4202BFBFF32F8F00200DE0C3891A44DE
:10BEA00083899A4228BFD21AC4EA024240E8022398
:10BEB000002BE8D14FF0010001948DF800000198AB
:10BEC00008609DF8000016BC7047000050E8022F83
:10BED000C2EA224240E802210029F7D1704700005F
:10BEE00070B4002901D10E2013E01400A4B21D008B
:10BEF000ADB294FBF5F605FB1644002C01D00920E9
:10BF000007E0016000214160002181608281C381DE
:10BF1000002070BC704738B504000D0029002000D7
:10BF2000FFF784FF002803D020682988084400E038
:10BF3000002032BD80B50A8849888A4203D1FFF7C4
:10BF400097FF012000E0002002BD38B504000D007D
:10BF500029002000FFF796FF002803D02068698899
:10BF6000084400E0002032BD80B50A8849888A4232
:10BF700003D1FFF7ABFF012000E0002002BDFEE788
:10BF8000BFF34F8F0548016811F4E0610448014395
:10BF900002480160BFF34F8F00BFFDE70CED00E0EA
:10BFA0000400FA0580B572B6FDF74CFEFDF7A1FC62
:10BFB0000028FBD10D490E480E4A801AC008000423
:10BFC00050F00100FDF773FC0B480068C00700D576
:10BFD00000BE0A490648074A801AC008000450F00B
:10BFE0000200FDF764FCFFF7CBFF01BD4C0D030021
:10BFF000B4FE02008CFE0200F0ED00E0100C030025
:10C0000000B500BF130096469446103928BFA0E83B
:10C010000C50FAD85FEA417C28BF0CC048BF40F8FA
:10C02000042BC90728BF20F8022B48BF00F8012BBA
:10C0300000BDFEE7012210F01F018A40DFF87416F0
:10C0400040B2400941F820207047020052B2002A55
:10C0500009D54901DFF8602640B210F00F00104406
:10C0600000F8041C04E04901DFF8502640B21154E6
:10C07000704710F06040B0F1005F01D1012000E096
:10C080000020C0B27047000B40B2704780B5C9B203
:10C0900040B2FFF7DAFF01BD80B540B2FFF7CAFF3B
:10C0A00001BD81B000220B001BB2C25009B2405842
:10C0B0000090009801B0704709B24058002801D0A4
:10C0C000012000E00020C0B27047D0F800221143E8
:10C0D000C0F800127047D0F8002232EA0101C0F81F
:10C0E00000127047C0F804137047C0F80813704777
:10C0F0000100D1F88004C1F8800470470821C0F81D
:10C1000000157047C0F80C15C0F814257047C0F82A
:10C110000815C0F8102570470122C9B24250704777
:10C12000C9B2D2B21143C0F86C157047C0F82415DB
:10C130007047C0F84415C0F848257047D0F84C0542
:10C140007047C0F83415C0F838257047D0F83C0562
:10C1500070475FF0A04070472DE9F14181B00E00BB
:10C1600017009846089D099C01A8FFF7F2FFF6B258
:10C17000FFB256EA47065FFA88F856EA8806EDB23B
:10C1800056EA0526E4B256EA0446019900EB81001E
:10C19000C0F80067BDE8F381E0B5002101910021FE
:10C1A0000091002301220121FFF7D6FF07BDE0B572
:10C1B0000B000021019100210091DBB2002200213F
:10C1C000FFF7CAFF07BD01B56846FFF7C2FF0121AF
:10C1D000009A914000F001F801BDC0F808157047C1
:10C1E00038B504000D00286810F1010F05D028684B
:10C1F000FFF7E9FF2868FFF7CFFF686810F1010F2C
:10C2000003D000216868FFF7D2FFA9692068FFF713
:10C210008DFF2A7D697D2068FFF782FF6A682968A3
:10C220002068FFF76FFF287D012816D1A86810F15C
:10C23000010F03D00021A868FFF7B9FFE86810F1EB
:10C24000010F05D0E868FFF7BEFFE868FFF7A4FF1D
:10C25000AA68E9682068FFF75AFF31BD38B50400C5
:10C260000D004FF488712068FFF71BFF4FF49071A9
:10C270002068FFF716FF4FF492712068FFF711FF57
:10C280004FF4A2712068FFF70CFF4FF4AC712068E7
:10C29000FFF707FFDFF828142068FFF723FF206867
:10C2A000FFF7F1FE2900C9B240B2FFF7EFFE2068A8
:10C2B000FFF7E9FE40B2FFF7EFFE31BD2DE9F04197
:10C2C00004000D001600DFF8FC13227924204243FD
:10C2D00001EB02075FF0000897F82000002801D06A
:10C2E000082026E0DFF8E003217950F821102068CB
:10C2F00001F04AFE002801D011201AE02900200098
:10C30000FFF76EFF7E60286938607868002803D0E8
:10C31000297F2000FFF7A2FF2068FFF7EFFE002033
:10C32000B8610020F86100207861012087F82000C2
:10C330004046BDE8F081F8B505000C001700DFF8B5
:10C3400084132A792420424301EB02062000FFF7E0
:10C3500090FE002801D1102044E0280000F043F8AE
:10C36000002801D011203DE07761B46000274FF430
:10C3700090712868FFF795FE4FF4AC712868FFF7BD
:10C3800090FE7269B1682868FFF7D3FE082128681B
:10C39000FFF7C2FE7068002823D14FF4907128681F
:10C3A000FFF78AFE04004FF4AC712868FFF784FEA3
:10C3B000E4B2002C03D10100C9B20029EDD0C0B213
:10C3C000002801D00F270AE00C212868FFF7A4FEFF
:10C3D0004FF4AC712868FFF76FFE0028F8D00020FA
:10C3E00070613800F2BDDFF8DC120279242042438C
:10C3F00001EB02004069002801D0012000E000208C
:10C40000C0B270472DE9F04106000D009046AD49DD
:10C4100032792420424301EB02072800FFF729FE6E
:10C42000002801D110207EE000247868002804D084
:10C430004FF404713068FFF758FEB86900280DD03A
:10C44000F869002809D07868002804D04FF40471F6
:10C450003068FFF747FE112065E001242000C0B2DC
:10C46000002805D1C7F81880FD600020F86102E0BF
:10C470003D61C7F81C8000274FF488713068FFF7D2
:10C4800010FE4FF4A2713068FFF70BFE4246290000
:10C490003068FFF756FEE4B2002C04D1002130686A
:10C4A000FFF73AFE03E020213068FFF70EFE8549D2
:10C4B00032792420424301EB0200406800282CD14D
:10C4C0004FF488713068FFF7F7FD04004FF4A27154
:10C4D0003068FFF7F1FD05004FF492713068FFF707
:10C4E000EBFDE4B2002C07D12900C9B2002903D129
:10C4F0000100C9B20029E3D0724A337924214B43A9
:10C5000002EB030100228A61C0B2002800D0032799
:10C51000EDB2002D06D00F2704E04FF4047130680F
:10C52000FFF7E0FD3800BDE8F081F8B50300012019
:10C530008DF8000002910192196868465A68904788
:10C5400005B000BDF8B5020000208DF80000029192
:10C5500090680190002050611168684652689047C9
:10C5600005B000BDF8B584B005000C004FF4927121
:10C570002800FFF7A1FD00281AD04FF4927128007F
:10C58000FFF78FFD02208DF800002800FFF7B0FDB7
:10C5900003902800FFF7DAFD0290E0680190002088
:10C5A000A0610020E06121686846626890472DE044
:10C5B0004FF488712800FFF77FFD002826D04FF444
:10C5C00088712800FFF76DFD2800FFF7BFFD06000A
:10C5D000A06986421AD1E069002810D0E7682021BE
:10C5E0002800FFF778FDE069A0612069E060002085
:10C5F000E0613A0031002000FFF797FF06E00020DD
:10C60000A061E26831002000FFF78FFF4FF4A271B4
:10C610002800FFF751FD002813D04FF4A271280025
:10C62000FFF73FFDA06900280BD00020A06100208B
:10C63000E0612800FFF78AFDE26801002000FFF7B3
:10C6400074FF4FF490712800FFF736FD002812D0D8
:10C650004FF490712800FFF724FD0C212800FFF70C
:10C660005BFD6069002806D02800FFF767FD010028
:10C670002000FFF767FF4FF4AC712800FFF71CFDA7
:10C6800000280ED04FF4AC712800FFF70AFD606956
:10C69000002806D02800FFF751FD01002000FFF719
:10C6A00051FF05B0F0BD80B506490848FFF75AFFB5
:10C6B00001BD000000E100E018ED00E000E400E052
:10C6C00010034200E03E0020A80F030000200040BD
:10C6D000012210F01F018A40DFF8001740B2400924
:10C6E00041F820207047020052B2002A09D54901C2
:10C6F000DFF8EC2640B210F00F00104400F8041CE4
:10C7000004E04901DFF8DC2640B211547047000B09
:10C7100040B2704780B5C9B240B2FFF7E4FF01BD37
:10C7200080B540B2FFF7D4FF01BD81B000220B00FD
:10C730001BB2C25009B240580090009801B0704737
:10C7400009B24058002801D0012000E00020C0B20A
:10C750007047C0F804137047D0F80403084201D0B2
:10C76000012000E00020C0B27047C0F808137047F5
:10C770000100D1F88004C1F8800470470421C0F89A
:10C7800000157047C0F81425C0F80C157047C0F8A4
:10C790000815C0F810257047D0F81805C0B27047CA
:10C7A000C9B2C0F81C1570470122C9B24250704787
:10C7B000C9B2D2B21143C0F86C157047C0F8241545
:10C7C00070475FF0A04070472DE9F14181B00E0045
:10C7D00017009846089D099C01A8FFF7F2FFF6B2E2
:10C7E000FFB256EA47065FFA88F856EA8806EDB2C5
:10C7F00056EA0526E4B256EA0446019900EB8100A8
:10C80000C0F80067BDE8F381E0B500210191002187
:10C810000091002301220121FFF7D6FF07BDE0B5FB
:10C820000B000021019100210091DBB200220021C8
:10C83000FFF7CAFF07BD01B56846FFF7C2FF012138
:10C84000009A914000F001F801BDC0F8081570474A
:10C8500038B504000D00286810F1010F05D02868D4
:10C86000FFF7E9FF2868FFF7CFFF686810F1010FB5
:10C8700003D000216868FFF7D2FFA9692068FFF79D
:10C880009DFF2A7D697D2068FFF792FF6A6829680D
:10C890002068FFF777FF287D012816D1A86810F1DE
:10C8A000010F03D00021A868FFF7B9FFE86810F175
:10C8B000010F05D0E868FFF7BEFFE868FFF7A4FFA7
:10C8C000AA68E9682068FFF762FF31BD38B5040047
:10C8D0000D004FF48E712068FFF727FF4FF4A2710F
:10C8E0002068FFF722FFDFF800152068FFF731FF0F
:10C8F0002068FFF70CFF2900C9B240B2FFF70AFF1A
:10C900002068FFF704FF40B2FFF70AFF31BD2DE9B1
:10C91000F04104000D001600DFF8D01422792C201D
:10C92000424301EB02075FF0000897F82A00002855
:10C9300001D0082029E0DFF8B804217950F821104F
:10C94000206801F021FB002801D011201DE0290002
:10C950002000FFF77DFF7E60286938607868002836
:10C9600003D0297F2000FFF7B1FF2068FFF706FF03
:10C970000020B8610020F861002087F8290000201D
:10C980007861012087F82A004046BDE8F08138B57B
:10C9900004000D004FF48E712000FFF7C6FEA8685A
:10C9A000296A415C286A401C2862C9B22000FFF74E
:10C9B000F7FE31BD70B504000D006E6903E029007B
:10C9C0002000FFF7E4FF286AB0420CD24FF48E71CA
:10C9D0002000FFF7B5FE0028F1D195F828000028C7
:10C9E000F4D0002000E0012070BDF8B504000E0076
:10C9F0001700DFF8F81322792C20424301EB0205DF
:10CA0000200000F033F8002801D011202DE06F61E4
:10CA1000AE6000202862002085F8280000264FF430
:10CA20008E712068FFF781FE08212068FFF7BCFEA9
:10CA300029002068FFF7ABFF6868002814D129009F
:10CA40002068FFF7B7FF002801D10F260AE04FF456
:10CA50008E712068FFF774FE0028F8D00C21206842
:10CA6000FFF7A2FE002068613000F2BDDFF87C1302
:10CA700002792C20424301EB02004069002801D0DA
:10CA8000012000E00020C0B2704710B504004FF450
:10CA900092712068FFF749FE4FF484712068FFF718
:10CAA00044FE00212068FFF77FFE10BD70B5040032
:10CAB0000D00A869002808D14FF484712000FFF709
:10CAC00034FE2000FFF768FE0DE04FF48471200073
:10CAD000FFF72BFE6E6A2000FFF75EFEE9688855BF
:10CAE000686A401C686270BD2DE9F04107000D00C6
:10CAF0001600DFF8F8123A792C20424301EB0208C5
:10CB00000024D8F80400002804D04FF401713868DC
:10CB1000FFF72BFED8F8180000280FD0D8F81C001B
:10CB200000280AD0D8F80400002804D04FF401717E
:10CB30003868FFF70EFE112077E001242000C0B214
:10CB400000280AD1C8F81860C8F80C500020C8F8AE
:10CB500024000020C8F81C0003E0C8F81050C8F8F2
:10CB60001C6098F82900002805D1E4B2002C02D1FD
:10CB70003800FFF78AFFD8F8040000284FD14FF49F
:10CB8000A2713868FFF7D1FD4FF492713868FFF752
:10CB9000D7FD05004FF484713868FFF7D1FD04001C
:10CBA0004FF4A2713868FFF7CBFD0600E4B2002C09
:10CBB00007D13000C0B2002803D12800C0B200283D
:10CBC000E2D02800C0B200280ED13000C0B2002848
:10CBD0000AD141463868FFF769FFD8F82400D8F831
:10CBE00018108842D0D3FFE70020C8F81800EDB233
:10CBF000002D01D0032018E0F6B2002E01D00F2046
:10CC000013E098F82900002804D000213868FFF7C5
:10CC1000CBFD09E004213868FFF7C6FD04E04FF4BE
:10CC200001713868FFF795FD0020BDE8F081F8B587
:10CC3000030001208DF800000291019219686846F6
:10CC40005A68904705B000BDF8B5020000208DF885
:10CC500000000291906801900020506111686846C0
:10CC60005268904705B000BD38B584B005000C008F
:10CC70004FF400712800FFF76FFD00282CD04FF40F
:10CC800092712800FFF75CFD002825D04FF49271C7
:10CC90002800FFF74AFD4FF401712800FFF765FDFA
:10CCA00094F82900002803D104212800FFF77CFD17
:10CCB00002208DF800002800FFF75AFD0390A069BC
:10CCC0000290E06801900020A0610020E0612168EE
:10CCD00068466268904739E004212800FFF73CFD70
:10CCE000002833D04FF484712800FFF729FD002875
:10CCF0002CD021002800FFF7D9FEA069616A884284
:10CD000024D1E06900280DD0E268616AE069A06181
:10CD10002069E0600020E061002060622000FFF7F1
:10CD200086FF13E094F82900002803D1042128008D
:10CD3000FFF73AFD4FF401712800FFF716FD0020C0
:10CD4000A061E268616A2000FFF771FF4FF48E7105
:10CD50002800FFF7F5FC002818D06069216A81429D
:10CD600008D294F82800002804D121002800FFF7F9
:10CD70000EFE0BE04FF48E712800FFF7D6FC6069C1
:10CD8000002803D061692000FFF75EFF4FF4A27115
:10CD90002800FFF7D5FC002816D04FF4A271280018
:10CDA000FFF7C3FC94F82900002803D000212800D5
:10CDB000FFF7FAFCA069002806D00020A061E26815
:10CDC000616A2000FFF733FF05B030BD80B5074929
:10CDD0000848FFF749FF01BD0000000000E100E046
:10CDE00018ED00E000E400E080000200B43E002006
:10CDF000A40F03000020004001008868C968081AD9
:10CE0000704710B40368C468828814401955C1681B
:10CE1000491CC16010BC704710B40368846814FAE0
:10CE200081F180880140585C107010BC704710B5CB
:10CE300004000A0000212000FFF7EEFFA068401C5C
:10CE4000A06010BD10B4002901D10E2014E0130021
:10CE50009BB2002B06D013009BB25B1E1400A4B241
:10CE6000234201D0092007E00160511E818000218A
:10CE700081600021C160002010BC704738B50400FB
:10CE80000D002000FFF7B8FFA188814206D32900DA
:10CE9000C9B22000FFF7B5FF002000E0042032BD3A
:10CEA00038B504000D002000FFF7A6FF002805D0CC
:10CEB00029002000FFF7BBFF002000E0052032BD65
:10CEC000F8B50A0001788DF8001041680191816879
:10CED0008DF80810C06803902A4850F82210684660
:10CEE000294B53F82220904705B000BDF8B50A0041
:10CEF00001788DF800104168019181688DF8081063
:10CF0000C06803901F4850F8221068461E4B53F823
:10CF10002220904705B000BD70B588B00400150010
:10CF20002678194840F826500869164A42F8260023
:10CF3000487F164A905568462022FAF75FFA049611
:10CF4000002012492278895C002909D0002D01D0E7
:10CF50000F4A00E000226946201DFFF7AFF90EE0FE
:10CF60000A492278895C002909D1002D01D0094A9B
:10CF700000E00022694614F10C00FFF7C8FC08B07D
:10CF800070BD0000C0400020BC400020D9400020FF
:10CF9000C1CE0200EDCE020080B501F024F802BD42
:10CFA0002DE9F04105002F8A3F1F7918C91CB1FBFC
:10CFB000F7F6280001F034F80400002C01D100201D
:10CFC00020E00020207101206071E7802700F6B288
:10CFD000761E3D605FF0000807E06179491C6171D1
:10CFE00038600560070018F10108B04509D2280033
:10CFF00001F016F80028F0D1200000F005F800201C
:10D0000000E02000BDE8F081F8B501004C790A008D
:10D010002300DBB25B1E002001E01268401C984236
:10D02000FBD31768002505E00E68380001F024F8EE
:10D0300031006D1C2000C0B28542F5D3F1BD80B532
:10D040000121001D00F0B8F801BD1CB5040001214C
:10D05000201D00F0BFF8009068460078002802D13B
:10D060002000FFF7D1FF13BD2DE9F84F0700C58859
:10D07000447965432D1FC688181DB0FBF6F01C1DB2
:10D08000B4FBF6FC06FB1C4C14681C19A54202D22A
:10D09000EB1A1C0000E01468146001E03F68401EB9
:10D0A0000028FBD10A9D88465FF00009B6EB0C0A08
:10D0B000544501D2A24601E000E0A246002C1FD058
:10D0C00008EB090107EB0C00001D2A00D2B2002A70
:10D0D00006D052468B4601005846FAF77FF904E025
:10D0E000524683465846FAF779F95FF0000C3F68DC
:10D0F000B4EB0A041AEB0909B442DED3B246DDE709
:10D10000BDE8F18FE0B501920022009201AAFFF77D
:10D11000ABFF07BDE0B501920122009201AAFFF723
:10D12000A3FF07BD00218268916000218268116120
:10D1300000218268516100218268D16000218268EB
:10D1400051600021806801607047FEE710B4020062
:10D1500052E8000F0B4642E8003494F0000FF7D17C
:10D1600010BC704710B4020052E8003F43EA0100CF
:10D1700042E8000494F0000FF6D110BC70470000A4
:10D1800010B4020052E8000F00EA010342E8003444
:10D1900094F0000FF6D110BC7047000010B40200EC
:10D1A00052E8003F03EA010042E8000494F0000F57
:10D1B000F6D110BC7047000010B4020052E8003FE6
:10D1C00003EB010042E8000494F0000FF6D110BC1C
:10D1D0007047000010B4020052E8003FA3EB0100CA
:10D1E00042E8000494F0000FF6D110BC704780B5FF
:10D1F0000121FFF7B7FF02BD80B50021FFF7C0FF97
:10D2000002BDFEE7EFF3108072B6704762B670475A
:10D2100010B50400FFF7F6FF1E498968002916D1F2
:10D2200001211C4A91601C490A681C490A4019499D
:10D230000A601A49184A116019490968154A51606B
:10D240005FF0FF31164A11600021217001E00121D9
:10D250002170002801D1FFF7D9FF002010BD80B553
:10D260000C498968002913D0C0B2002810D1FFF7FB
:10D27000C9FF084909680B4A1160064949680A4A0A
:10D2800011600021034A9160002801D1FFF7BEFF21
:10D29000002002BD1440002080E100E0FC06FFBD3C
:10D2A00084E100E000E100E004E100E080B5FFF788
:10D2B000AFFF01BD80B5C0B2FFF7D1FF01BD38B5EA
:10D2C00005001400002C01D10E202CE0002020606D
:10D2D000002D01D10E2026E02868002801D10E2063
:10D2E00021E0E888042290FBF2F302FB13000028FF
:10D2F00001D0072017E0080080B200F0BEFF010057
:10D30000C9B2142901D105200DE001002A79C9B262
:10D31000914201D3042006E02A68C0B2E98848435C
:10D3200010442060002032BD01000878497850EA9E
:10D33000012080B2704780B5FFF7F6FF10F00100C2
:10D3400002BD0A7812F0F0020A700A7812F00F0299
:10D350000A70C0B2002808D002281CD00ED30428BE
:10D3600033D025D305283DD048E0087810F0F000F0
:10D370000870087810F00F0008703FE0087810F08F
:10D38000F00050F001000870087810F00F0050F025
:10D390001000087032E0087810F0F00050F0010042
:10D3A0000870087810F00F0050F02000087025E099
:10D3B000087810F0F00050F001000870087810F0C4
:10D3C0000F0050F03000087018E0087810F0F000FE
:10D3D00050F002000870087810F00F0050F01000B4
:10D3E00008700BE0087810F0F00050F002000870B0
:10D3F000087810F00F0050F0200008707047F8B562
:10D4000090B004000D001600A878002803D1012078
:10D410008DF80E0002E0A8788DF80E002888ADF88F
:10D420000C000321002201AF3800FBF7B5FE01A973
:10D43000687CFFF786FF0DF10501A87CFFF781FFEF
:10D44000E87B002801D0012000E000209DF80610B4
:10D4500060F3C3018DF80610287C002801D001205C
:10D4600000E000209DF8061060F304118DF806100E
:10D47000287B002801D0012000E000209DF8061044
:10D4800060F300018DF80610287D002801D00220ED
:10D4900000E001209DF8061060F342018DF80610AF
:10D4A0001C21002209AF3800FBF776FE687B10F0E4
:10D4B000300F24D00321002202AF3800FBF76CFEAE
:10D4C0000DF10901E87CFFF73CFF9DF8080010F022
:10D4D000F00050F001008DF808009DF8080010F0F1
:10D4E0000F0050F010008DF808009DF80A0010F0B1
:10D4F000F90050F002008DF80A0002A80E90687B37
:10D500008DF82400A87B8DF825001421002204AF9B
:10D510003800FBF741FE03A8049001A80590A888F5
:10D52000ADF81C00A868002804D0E888ADF8180001
:10D53000A8680890A869002851D0032100226F46EE
:10D540003800FBF729FEA8690088ADF82C00A8690F
:10D550004088ADF82E00A86940680A9068460D9092
:10D560006946A869007BFFF7ECFE0DF10101A8698F
:10D57000407BFFF7E6FEA869807A002801D00120F1
:10D5800000E000209DF8021060F3C3018DF8021046
:10D59000A869C07A002801D0012000E000209DF891
:10D5A000021060F304118DF80210A869007A0028B7
:10D5B00001D0012000E000209DF8021060F300017E
:10D5C0008DF80210A869807B002801D0022000E0BD
:10D5D00001209DF8021060F342018DF80210E86905
:10D5E000002801D0E8690C90330004AA09A92000A2
:10D5F00080B2AADF11B0F0BD5FF0A040704701B566
:10D600006846FFF7F9FF0121009A914000F035F8D4
:10D6100001BD01B56846FFF7EFFF0121009A914077
:10D6200000F02EF801BD01B56846FFF7E5FFD0F820
:10D630000425012300998B409343C0F8083501234A
:10D6400000998B401A40C0F80C2501BD80B5002917
:10D6500002D1FFF7DEFF01E0FFF7D1FF01BD01B509
:10D660006846FFF7C9FF00F005F80099C84010F0C0
:10D67000010002BDD0F804057047C0F808157047D6
:10D68000C0F80C15704780B51C49085CFFF7E7FF30
:10D69000002801D0012000E0002090F00100C0B27D
:10D6A00002BD80B50021154A105CFFF7CFFF01BD18
:10D6B00080B50121114A105CFFF7C8FF01BD10B50C
:10D6C000002403E02000FFF7F3FF641C042CF9D3CF
:10D6D00010BD10B5002403E02000FFF7E2FF641C3A
:10D6E000042CF9D310BD80B50449085CFFF79BFFFB
:10D6F00001BD0349085C704700000000780F03007B
:10D700007C0F0300087080B2000A48700220704746
:10D710007CB504000D0092B228880930824201D203
:10D720000C202DE068466DDF002829D108202988CB
:10D7300060542888401C28801B2029886054288831
:10D74000401C288006220DF10101288804EB000608
:10D750003000F9F743FE2888801D28809DF80000DE
:10D76000C0B24008C0B2002803D10020298860540C
:10D7700002E00120298860542888401C288000206D
:10D7800076BD78B405000C002878012804D16878AB
:10D79000002801D107205AE0180080B21188891CA6
:10D7A00088420BD3287801280AD1180080B211884A
:10D7B0006E7816FA81F1891C884201D20C2046E06D
:10D7C0009BB210881B1A9B1EADF80030694610886A
:10D7D0002044801C7DDF002839D12878022805D01C
:10D7E0006878BDF8001080B2884207D31800BDF8F1
:10D7F000001080B2884201D309200FE00820297868
:10D80000012909D119006E7889B2B6B2B14203D3A9
:10D810006978ADF8001001E0ADF80030BDF80010F7
:10D82000FF2901D30C2012E0BDF80010491C138819
:10D83000E1541188491C1180118860541088401CE3
:10D8400010801188BDF8000041181180002072BCC2
:10D8500070471CB503000C0092B22088001D824264
:10D8600001D20C201BE0684679DF002817D1032085
:10D87000218858542088401C208019202188585421
:10D880002088401C2080208803EB0001BDF80000A8
:10D89000FFF738FF218851FA80F02080002016BD64
:10D8A00010B49BB21488E41CA34201D20C2011E0F6
:10D8B000022314880B5513885B1C138001231488E2
:10D8C0000B5513885B1C13801388C8541088401CA8
:10D8D0001080002010BC704710B49BB21488E41C68
:10D8E000A34201D20C2011E0022314880B551388A7
:10D8F0005B1C13800A2314880B5513885B1C138050
:10D900001388C8541088401C1080002010BC704739
:10D910002DE9FC4706000F0094461C00DDF828E0C6
:10D920000B9D0023BEF800805FF0000924E0180082
:10D93000C0B200280DD1BEF80000401CAEF80000B7
:10D94000BEF800002754BEF80000401CAEF80000EE
:10D950000123BEF8000004EB0002694601A864DF61
:10D96000002832D1BEF800009DF8001050FA81F076
:10D97000AEF8000019F101093088814526DA706897
:10D9800050F8291001910022694601A864DF00289F
:10D990000BD19DF800006146C9B28842EAD1180057
:10D9A000C0B2002802D0002101E023E002212800BB
:10D9B00080B2BEF800209DF800A01AFA82F252FA56
:10D9C00081F18842B3DA0C2014E013E0DBB2002BC3
:10D9D0000FD0BEF80000B0EB0800401E010089B275
:10D9E000B1F5807F01DB0C2004E01FFA88F804F811
:10D9F00008000020BDE8F6872DE9FC41050016006F
:10DA00001F00DDF82080099C200080B20190CDF835
:10DA100000803B000222C9B22800FFF779FF0028EE
:10DA20000DD1A4B20194CDF800803B00102231004A
:10DA3000C9B22800FFF76CFF002800D10020BDE824
:10DA4000F6810188062909DB018840F6814291426E
:10DA500006DB01884FF6FF72914201D007201FE0DC
:10DA60004188062909DB418840F68142914206DB64
:10DA700041884FF6FF72914201D0072010E00188E3
:10DA80004FF6FF7291420AD041884FF6FF729142E1
:10DA900005D041880088814201D2072000E00020A3
:10DAA000704770B505000E0014009BB22088801DE1
:10DAB000834201D20C2025E02800FFF7C2FF002896
:10DAC00020D10520218870542088401C20801220FD
:10DAD000218870542088401C2080208806EB00019B
:10DAE0002888FFF70FFE218851FA80F020802088D7
:10DAF00006EB00016888FFF705FE218851FA80F0E7
:10DB00002080002070BD70B504000E001500A088B4
:10DB1000801C9BB2298810FA81F1891C8B4201D2AA
:10DB20000C202DE0FF2801D30C2029E0401C29887F
:10DB300070542888401C2880FF2029887054288829
:10DB4000401C2880288806EB00012088FFF7DAFDBA
:10DB5000298851FA80F02880A08800280FD0A0687A
:10DB6000002801D107200BE0A288A168288806447C
:10DB70003000F9F733FC2988A0884118298000205B
:10DB800070BD2DE9F84304000F009046A06A0028FC
:10DB900001D107204CE0002534E0401CB8F800100B
:10DBA0007854B8F80000401CA8F800001620B8F817
:10DBB00000107854B8F80000401CA8F80000B8F82D
:10DBC000000007EB00013088FFF79CFDB8F800105B
:10DBD00051FA80F0A8F80000B088002811D0B06891
:10DBE000002822D0B288B168B8F8000007EB00091D
:10DBF0004846F9F7F3FBB8F80010B0884118A8F8C8
:10DC000000106D1C280094F82C10C0B288420ED26F
:10DC1000A16A2A00D2B20C20424301EB0206B0886E
:10DC2000801CFF28B9D30C2002E0072000E0002070
:10DC3000BDE8F283FEB504000D0016000020378811
:10DC40000021318094F82D10002908D03A0092B2BA
:10DC500031002800FFF75CFD002840F08880A178A3
:10DC6000002907D03A0092B231002800FFF7F1FDF9
:10DC700000287CD1E17800290AD03B009BB2320019
:10DC8000290094F9030040B2FFF70AFE00286ED184
:10DC9000616800290AD03B009BB23200290060680D
:10DCA00090F90000FFF718FE002860D121890029B3
:10DCB0000CD0380080B2019000962B000622022181
:10DCC00014F10800FFF798FE002850D1218A00299E
:10DCD0000CD0380080B2019000962B00072203215F
:10DCE00014F11000FFF788FE002840D1218B002995
:10DCF0000CD0380080B2019000962B001522142120
:10DD000014F11800FFF778FE002830D1216A0029AD
:10DD100008D03B009BB232002900206AFFF7C1FE09
:10DD2000002824D1616A002908D03B009BB2320050
:10DD30002900606AFFF7E7FE002818D194F82C103C
:10DD4000002908D03B009BB2320029002000FFF7D9
:10DD500018FF00280BD12178002908D03B009BB286
:10DD6000320029002000FFF70CFD0028FFD1FEBD86
:10DD700070B4002801D0002A01D1002030E0002436
:10DD800004E02500ADB2455D6D1C2C1925001688F8
:10DD9000ADB2B54207D32500ADB205446D781E0083
:10DDA000F6B2B54205D025000E00ADB2B6B2B5420E
:10DDB000E7D323000D009BB2ADB2AB4201D30020EC
:10DDC0000EE0A31CA4B2005D401E89B20400A4B200
:10DDD00014FA83F4A14201DA002001E0138080B23A
:10DDE00070BC70471CB5040013000020ADF80000A3
:10DDF000DBB26A4689B22000FFF7BAFF80B2002882
:10DE000001D1002002E0BDF80000204416BD08E06A
:10DE1000416809684268526891420AD141680831F4
:10DE200041604168026852689142F1D100218160ED
:10DE300002E0416809688160704780B50160096847
:10DE40004160FFF7E4FF01BD80B5816800290ED075
:10DE50008268016889688A188260816842685268AD
:10DE6000914204D1416808314160FFF7D0FF01BD04
:10DE700080B500F005F8002801D10F48FFE702BD8A
:10DE800010B40E490E4A00E01A00914210D2531A03
:10DE9000DB10022493FBF4F301EBC3031C68A042E4
:10DEA000F2D3844202D213F10801EEE7586800E091
:10DEB000002010BC70470000E80B0300E0FA0200ED
:10DEC00008FC020080B5002805D0224A52F0010269
:10DED00040214843904701BD10B50400002C06D0F6
:10DEE0004FF47A70FFF7EEFF641E002CF8D110BDDE
:10DEF00080B500F0BCFA01BDF8B50E001400002C8E
:10DF00001FD000270325220006EB0701002000F0A8
:10DF100079FAC719241A002809D10F480078002877
:10DF20000BD00120FFF7D8FF6D1E002D06D0012079
:10DF300009490870002CE6D103E002E00020064900
:10DF40000870F1BD80B5054A00924023044A00F0F4
:10DF50009DFA01BDA00E0300DA400020F9DE0200A8
:10DF6000743E00207047704780B5054800688047C0
:10DF700001BD0449884201D1014800E000207047FA
:10DF800080400020002000407CB50E00FFF7F1FF2C
:10DF90000500002D17D0002400208DF800006846F1
:10DFA000FFF784F92879002801D0012402E02E60CF
:10DFB000012028719DF80000FFF77CF9E4B2002CE5
:10DFC00001D0112000E0002076BDC268C9B2008AED
:10DFD000414302EB01007047C268891A008AB1FB15
:10DFE000F0F0C0B2704710B4002801D10E2015E047
:10DFF000816842688A1A41680368196005E001680F
:10E0000009684B1C046823600A7011004A1EC9B2DB
:10E010000029F4D1002100680171002010BC704774
:10E0200038B50400002500208DF800006846FFF791
:10E030003DF9606821680968884217D22068006845
:10E04000401E216808602068006801782000FFF702
:10E05000BCFF0500A16820680068081A21680979DA
:10E060000200D2B2914201D2216808719DF80000ED
:10E07000FFF720F9280032BD7CB504000D00002018
:10E080008DF800006846FFF711F920680668701CDB
:10E090002168086029002000FFF79EFF30709DF87E
:10E0A0000000FFF707F973BD33B58BB00400002003
:10E0B00000900C98002812D000250EE029000CA832
:10E0C00000F067FA002807D06846009900EB41008D
:10E0D00085800098401C00906D1C142DEED320000C
:10E0E00069462C22F9F78AF90DB030BD10B504004D
:10E0F000200080B2142801DB00200CE0210089B24E
:10E10000DFF8940100F02CFAA4B22100DFF88C01B2
:10E1100000F026FA012010BD38B50400002509E002
:10E12000210089B2DFF86C0100EB8500001D00F0D2
:10E1300023FA6D1C1E2DF3D331BD80B5010089B2C9
:10E14000DFF8540100F018FA01BD10B58CB0DFF80B
:10E1500044018068C0430090DFF838014168684698
:10E16000FFF71CF8009901A8FFF79EFF002406E0C6
:10E1700001A800EB44008088FFF7CEFF641C0198E3
:10E180008442F5D30CB010BD80B5D2B2002A03D0C2
:10E1900089B200F0E5F902E089B200F0EDF901BDC5
:10E1A00038B50500AC882888102806D0112819D069
:10E1B000192846D01A281AD051E0FFF7C6FF2000D0
:10E1C00080B2FFF793FF002803D10420FAF7B0FFD5
:10E1D00007E0E87B012804D0A4B22100304800F019
:10E1E000BFF93CE0200080B2FFF7A7FF37E02D7AAF
:10E1F000EDB22D092800C0B2042801DB012200E0A5
:10E200000022D2B2210089B22648FFF7BDFF2800C4
:10E21000C0B2032801DB012200E00022D2B22100BB
:10E2200089B22148FFF7B0FFEDB2022D01DB0122D8
:10E2300000E00022D2B2210089B21C48FFF7A4FFFF
:10E240000DE0287A00280AD1687AC0F3C00212F0E3
:10E250000102D2B2210089B21248FFF795FF31BD09
:10E2600080B5010089B2142901DB002004E080B2EE
:10E2700001000A4800F08DF902BD10B5040020002D
:10E2800080B2FFF7EDFF002802D0200080B200E04E
:10E29000142010BD2C3C0020343C0020303C0020D9
:10E2A000383C0020443C0020403C00203C3C002006
:10E2B00010B5DFF8C4410220206102206061DFF860
:10E2C000BC01A061DFF8B801E0614FF4007020628A
:10E2D0000020A062002060620020E062DFF89C0164
:10E2E000A064DFF8A001E064102020650020A06594
:10E2F000002060650020E06541A1E01D00F054F9B8
:10E30000DFF88411200000F04FF92020A07110BD2B
:10E310002DE9F04705000E0014000027D5F80C8009
:10E320002869804505D28146B9EB0809B9F1010990
:10E3300007E0D5F80890B9EB080910EB0909B9F125
:10E340000109A868B0EB0800814503D3D5F808900F
:10E35000B9EB0809A14500D3A146686800EB080A9B
:10E360004A4631005046F9F739F819EB07074E4491
:10E37000B4EB090419EB0809C846A868804501D127
:10E380005FF00008C5F80C80002CC9D13800BDE84A
:10E39000F0872DE9F04104000E001500D4F80C8040
:10E3A000A768B7EB0807BD420BD2606800EB08070F
:10E3B0002A0031003800F9F711F815EB0805E5607F
:10E3C0000FE0606880443A0031004046F9F706F8F3
:10E3D000ED1B06EB070166682A003000F8F7FEFF28
:10E3E000E560BDE8F08101000869CA68824204D393
:10E3F0008968491E8A1A801801E0801A401E7047F9
:10E400005254540070B50D001400DFF86C20182130
:10E410004843104410F118067069002803D0022800
:10E420001BD00DD320E03000FFF7DDFFA04201D26A
:10E43000002404E0220029003000FFF7AAFF14E0C6
:10E440003000FFF7D0FFA04201D20400FFE7220016
:10E4500029003000FFF79DFF07E02200290030006F
:10E46000FFF756FF040000E00024200070BD80B5D7
:10E47000FFF71EFF01BD0000A83C0020240E030092
:10E48000F835002004400020400F0300F0B595B09F
:10E490000D0016001F001A9C2800FEF7D0FD09A8E9
:10E4A0001821FAF755FE09960A970E9400230822C0
:10E4B00001A92800FEF72EFE082603980490BDF857
:10E4C0000800ADF81400BDF80A00ADF816000020F1
:10E4D0008DF81900019810F0030001281AD1019C51
:10E4E000A40A0198C0F3C2008DF818000198C0F387
:10E4F00083173300BA000FA92800FEF70BFE16EBB6
:10E50000870609A8009004AB3A000FA9200000F08C
:10E51000C2F820E0019810F0030002281BD1019CF2
:10E52000A40D0198C0F3C2008DF81800082C01D288
:10E53000270000E0082733003A0007A92800FEF76B
:10E54000E9FDBE19E41B09AB04AA390007A800F0D5
:10E5500021F9002CEAD12800FEF777FD15B0F0BDB7
:10E5600080B50B00012113F01F0291405B0900EB05
:10E570008300FEF7F7FD01BD80B50B00012113F00C
:10E580001F029140C9435B0900EB8300FEF706FEC2
:10E5900001BD0A00520950F8220011F01F01C840C5
:10E5A00010F001007047FEE75FEA000C80EA01030B
:10E5B0009B0715D1830706D011F8013B00F8013BFA
:10E5C000B3B18307F8D10A68B2F1013323EA020339
:10E5D00013F0803F02BF40F8042B51F8042FF3E7FB
:10E5E00011F8013B00F8013B13B111F8013BF9E7C9
:10E5F00060467047704738B504000D00E088002879
:10E6000007D096480090E388954A9649280000F084
:10E6100040F9207A05281FD0607A00280BD0217A93
:10E62000A088FAF7C9FF9049C0B251F8202085A10F
:10E63000280000F02EF921682800FFF7DBFF0021F9
:10E64000A088FAF7A9FF03008848217A50F8212012
:10E650008749280000F01DF931BD10B50C00017A82
:10E6600005290DD0407A002805D07F48026875A1A1
:10E67000200000F00EF974A1200000F00AF906E075
:10E68000D2B2002A03D070A1200000F002F92000CD
:10E6900000F0F2F810BD2DE9F84384B00700884679
:10E6A00091461C000C9D2E7B002028732900200021
:10E6B000FFF7A1FFB9F1000F0CD0B9F1020F15D08F
:10E6C0000DD3B9F1040F26D019D3B9F1060F43D0F9
:10E6D00030D356E03900280000F0DBF851E0D8F8DC
:10E6E00000203900280000F0D4F84AE0D8F80430BF
:10E6F000D8F800203900280000F0CBF841E0D8F825
:10E7000008000090D8F80430D8F80020390028001C
:10E7100000F0BFF835E0D8F80C000190D8F80800F8
:10E720000090D8F80430D8F800203900280000F014
:10E73000B0F826E0D8F810000290D8F80C0001904C
:10E74000D8F808000090D8F80430D8F80020390034
:10E75000280000F09EF814E0D8F814000390D8F8D0
:10E7600010000290D8F80C000190D8F80800009032
:10E77000D8F80430D8F800203900280000F089F8D3
:10E78000FFE7002229002000FFF767FF2E7305B086
:10E79000BDE8F0832DE9F04706000C00170098460D
:10E7A000092C4DD298F80C50002088F80C004146F6
:10E7B0003800FFF720FF5FF000090EE023A140467C
:10E7C00000F067F807E0A145F8D216F809202949BA
:10E7D000404600F05EF819F10109B9F1080FF2D3D3
:10E7E0001BA1404600F055F85FF000090DE019A1AB
:10E7F000404600F04EF806E05FF02E0A524616A1A1
:10E80000404600F046F819F10109B9F1080F10D29D
:10E81000A145ECD216F809A05046C0B27F28EBDA29
:10E820005046C0B200F046F80028E5D05FFA8AFAF8
:10E83000E4E7012241463800FFF70FFF88F80C504B
:10E84000BDE8F087257300000D0A0000202020009D
:10E850007C0000002000000025630000C80E0300BB
:10E86000D80E0300B8090300FC2B0020E82B002081
:10E87000940D0300100F030010B50400A0680028D9
:10E8800006D0A26821682069636998470020A060CB
:10E8900010BD0CB480B5002907D0054A126800925B
:10E8A00002AA00926A4600F025F901BC5DF80CFB53
:10E8B0008C0F030010B50446A4F120005F280BD391
:10E8C000204600F008FA38B9204600F00EFA401E43
:10E8D0008041C043C00F10BD012010BD38B50400F9
:10E8E0000D002800C0B20A2803D10D212000FFF737
:10E8F000F5FFA068411CA16021680D54A068616803
:10E90000884202D32000FFF7B7FF31BDF8B50600FB
:10E910000D0014000027D8070CD4002D1ED02800AD
:10E92000F8F70AFD070019E06D1C7F1CC9B2300022
:10E93000FFF7D4FF29780800C0B20028F4D1A7421D
:10E940001CD2002C1AD0641E20213000FFF7C6FF15
:10E95000F5E7641E20213000FFF7C0FFA74201D277
:10E96000002CF6D129780800C0B2002806D06D1C12
:10E970007F1CC9B23000FFF7B1FFF3E7F1BD2DE90D
:10E98000F84F0F00904639005FF0010903E0B1FB3A
:10E99000F8F119F101094145F9D21E00B14500D243
:10E9A000B146DDF82CA00A9C83465FEACA7014D4F5
:10E9B000002C12D05FEA8A7003D5002E01D13025D9
:10E9C00007E0202505E0641E2900C9B25846FFF77C
:10E9D00085FF002C01D0A145F5D3012502E0761E6C
:10E9E00008FB05F5022EFAD2B7FBF5F04045F7D249
:10E9F000B7FBF5F005FB10770C49095C5846FFF7AB
:10EA00006DFFB5FBF8F5002DF2D15FEACA700BD5AA
:10EA1000002C05D108E0641E20215846FFF75EFF58
:10EA2000002C01D0A145F6D3BDE8F18F800C030086
:10EA30002DE9FC4706000F0091461D00002F01D56F
:10EA4000784200E038005FF0010803E090FBF9F045
:10EA500018F101084845F9DAA84500D2A846DDF8C2
:10EA60002CA00A9C002C05D0002F02D45FEA4A702B
:10EA700000D5641E5FEA8A7001D5002D0ED05FEAD2
:10EA8000CA700BD4002C05D108E0641E2021300090
:10EA9000FFF724FF002C01D0A045F6D3002F05D5A9
:10EAA0007F422D213000FFF719FF06E05FEA4A7030
:10EAB00003D52B213000FFF711FF1AF003000228C5
:10EAC0000DD1002D0BD1002C05D108E0641E3021A2
:10EAD0003000FFF703FF002C01D0A045F6D3CDF89E
:10EAE00004A000942B004A4639003000FFF747FF8E
:10EAF000BDE8F387FEB50C00002C00F0EB8015009C
:10EB000006002178641C0800C0B2002814D0080058
:10EB1000C0B2252840F0D0800022012021780B00CF
:10EB2000DBB22B2B0DD02D2B02D0302B05D00CE0DF
:10EB300052F00102641C09E0C6E052F00202641CBB
:10EB400004E052F00402641C00E000200028E5D13B
:10EB500000200CE021780B00DBB2303B0A2B13D2F3
:10EB6000641C0A230F00FFB2303F03FB0070C9B2E0
:10EB70002A29EFD129682960296809682B681B1D9B
:10EB80002B600818641CFFE700232178C9B22E29E6
:10EB90000ED1641C06E0641C0A27C9B2303907FB99
:10EBA00003110B0021780F00FFB2303F0A2FF2D380
:10EBB000217801E0641C21780F00FFB26C2FF9D09E
:10EBC0000F00FFB2682FF5D0C9B225296DD05829A2
:10EBD00036D063290CD0642916D0692914D0702945
:10EBE00049D073293AD075291CD0782928D061E002
:10EBF00028682860286801682868001D2860C9B254
:10EC00003000FFF76BFE55E0296829602968096824
:10EC10002F683F1D2F60019200900A223000FFF7FD
:10EC200007FF47E029682960296809682F683F1DA8
:10EC30002F60019200900A223000FFF7A0FE39E019
:10EC400029682960296809682F683F1D2F60019293
:10EC5000009010223000FFF792FE2BE02968296017
:10EC6000296809682B681B1D2B6013000200300007
:10EC7000FFF74CFE1EE028682860286807682868AF
:10EC8000001D286030213000FFF728FE7821300079
:10EC9000FFF724FE00200190082000900823102296
:10ECA00039003000FFF76BFE04E025213000FFF74C
:10ECB00015FEFFE7641C03E0C9B23000FFF70EFE4B
:10ECC000207800287FF41DAF307B002802D0300070
:10ECD000FFF7D2FDF7BD10B50446F8F7B8FA0146C4
:10ECE00020460969BDE81040084710B50446F8F70A
:10ECF000AEFA01462046C969BDE810400847FEE764
:10ED0000BFF34F8FDFF8E404016811F4E061DFF82E
:10ED1000E0040143DFF8D4040160BFF34F8F00BF6C
:10ED2000FDE7DFF8D004DFF8D0140860704780B545
:10ED300000F026F9002807D0DFF8C0040068C0F30F
:10ED40000420DFF8BC14086000F044F9002804D067
:10ED5000DFF8B004DFF8B014086000F053F90028C1
:10ED600007D0DFF8A8040068C0F34230DFF8A01431
:10ED7000086000F06CF9002807D0DFF898040068FC
:10ED800030F08070DFF88C14086000F075F900280E
:10ED90000BD00020DFF8801408600020DFF87C141E
:10EDA00008600020DFF87814086000F08AF9002875
:10EDB00003D00320DFF86C14086000F097F90028F6
:10EDC0000FD00520DFF8601408600120DFF85C1424
:10EDD00008600020DFF8581408603F20DFF8541462
:10EDE000086000F098F9002865D0DFF84C0400684E
:10EDF000DFF848140860DFF848040068DFF84414BE
:10EE00000860DFF844040068DFF840140860DFF8A9
:10EE100040040068DFF83C140860DFF83C04006838
:10EE2000DFF838140860DFF838040068DFF83414BD
:10EE30000860DFF834040068DFF830140860DFF899
:10EE400030040068DFF82C140860DFF82C04006838
:10EE5000DFF828140860DFF828040068DFF82414BD
:10EE60000860DFF824040068DFF820140860DFF889
:10EE700020040068DFF81C140860DFF81C04006838
:10EE8000DFF818140860DFF818040068DFF81414BD
:10EE90000860DFF814040068DFF810140860DFF879
:10EEA00010040068DFF80C140860DFF80C04006838
:10EEB000DFF80814086000F043F9002807D0DFF8F5
:10EEC0000004006810F04F00DFF8F813086000F04D
:10EED0005CF9002809D0DFF8F0030068C00704D50A
:10EEE0007FF00100DFF8E013086000F073F90028FC
:10EEF00007D0DFF8D803006850F48060DFF8CC1347
:10EF00000860DFF8CC03006850F47000DFF8C0132D
:10EF10000860BFF34F8FBFF36F8FDFF8B80300684F
:10EF2000002804D4DFF8B0030068002825D50120AC
:10EF3000DFF8A8130860DFF8A80300680028FAD0FB
:10EF40001520DFF890130860DFF8940300680028AC
:10EF5000FAD01520DFF880130860DFF8840300681A
:10EF60000028FAD00020DFF874130860DFF870037F
:10EF700000680028FAD0FFF7C3FEFFF7D2FE01BDFC
:10EF8000DFF86003007800F0FF00062820D1DFF8EA
:10EF90005803007810F00F0F1AD1DFF850030078F3
:10EFA00010F0F000302801D1012012E0DFF83C031E
:10EFB000007810F0F000402801D1012009E0DFF8CE
:10EFC0002C03007810F0F000502801D1012000E05F
:10EFD00000207047DFF80C03007800F0FF000628DF
:10EFE0000ED1DFF80403007810F00F0F08D1DFF81E
:10EFF000FC02007810F0F000302801D1012000E080
:10F0000000207047B748007800F0FF0006281CD1A8
:10F01000B548007810F00F0F17D1B448007810F001
:10F02000F000302801D1012010E0B048007810F045
:10F03000F000402801D1012008E0AC48007810F031
:10F04000F000502801D1012000E000207047A548C1
:10F05000007800F0FF0006280CD1A348007810F0DB
:10F060000F0F07D1A148007810F0F000302801D12F
:10F07000012000E0002070479A48007800F0FF006F
:10F0800006281CD19848007810F00F0F17D1974828
:10F09000007810F0F000302801D1012010E09348F2
:10F0A000007810F0F000402801D1012008E08F48DE
:10F0B000007810F0F000502801D1012000E000207D
:10F0C00070478848007800F0FF0006280CD1864879
:10F0D000007810F00F0F07D18448007810F0F0008E
:10F0E000302801D1012000E0002070477D480078E1
:10F0F00000F0FF0006280CD17B48007810F00F0FBD
:10F1000007D17A48007810F0F000302801D10120B2
:10F1100000E0002070477348007800F0FF000628E8
:10F120000CD17148007810F00F0F07D16F480078AC
:10F1300010F0F000502801D1012000E000207047BD
:10F140006848007800F0FF0006281CD16648007867
:10F1500010F00F0F17D16548007810F0F00030283C
:10F1600001D1012010E06148007810F0F000402843
:10F1700001D1012008E05D48007810F0F00050282F
:10F1800001D1012000E0002070475648007800F0CF
:10F19000FF0006281CD15448007810F00F0F17D13B
:10F1A0005248007810F0F000302801D1012010E022
:10F1B0004E48007810F0F000402801D1012008E00E
:10F1C0004A48007810F0F000502801D1012000E0FA
:10F1D0000020704746480068062805D14548006869
:10F1E000062801D1012000E0002070470CED00E06E
:10F1F0000400FA050090D003202C00202403001006
:10F20000403501400DF0ADBA74C007404402001013
:10F210003C050040FCED00E00C0100401001004006
:10F2200038050040A00500401056004088560040B8
:10F2300018560040145600400404001020C5004039
:10F240000804001024C500400C04001028C500402C
:10F25000100400102CC500401404001030C50040FC
:10F260001804001034C500401C04001040C50040C4
:10F270002004001044C500402404001048C500408C
:10F28000280400104CC500402C04001050C500405C
:10F290003004001054C500403404001060C5004024
:10F2A0003804001064C500403C04001068C50040EC
:10F2B000400400106CC500404404001070C50040BC
:10F2C00058020010E40E0040000400403C170040CB
:10F2D00088ED00E0001200100412001004E5014067
:10F2E00000E40140E00F00F0E40F00F0E80F00F050
:10F2F000300100103401001080B500B200F018F8A1
:10F300000068012801D1012000E00020C0B202BD48
:10F310001CB50400200000B200F00AF800210160D2
:10F32000200000B200F004F800680090009813BDBF
:10F3300000B200F1804010F5C0407047DFF8E812DD
:10F34000096808407047DFF8E41251F82000C0F364
:10F3500004207047DFF8D41251F82000000C10F0A0
:10F36000030070475FF0A040704711B581B00C00FA
:10F3700001A8FFF7F7FF019900EB8101D1F8001711
:10F3800031F44031019A00EB8202C2F80017019972
:10F3900000EB8101D1F80017E4B251EA0441019A6F
:10F3A00000EB8200C0F8001713BD01B56846FFF7F7
:10F3B000D9FF009900EB8100D0F80007000C10F095
:10F3C000030002BDD0F810057047F8B504000D0029
:10F3D00016006846DFF858120A680260270007E046
:10F3E000684650F82700FFF7EDFF3060361D7F1CA0
:10F3F00028198742F4D3F1BD0200D20810F00700AB
:10F40000012313FA00F0895C0840704710B4020031
:10F41000D20810F007008B5C012414FA00F01843A6
:10F42000885410BC7047DFF80C12084490F9300083
:10F430007047DFF8001251F8200070472DE9F843BB
:10F4400084B000246846002101604FF480760127D3
:10F45000002512E0300000B2FFF74EFF002809D06F
:10F460003800FFF76BFF002804D0300000B2FFF730
:10F470004FFF3C437F00361D6D1C082DEAD34FF42F
:10F48000BE70FFF739FF00280AD04FF4BE70FFF7B7
:10F490003FFF54F000446A4601210020FFF795FF2A
:10F4A00020061BD00126002516E0264212D0280097
:10F4B000FFF749FF07002800FFF74CFF80462800B0
:10F4C000FFF7B7FF02001000002803D04146C9B281
:10F4D0003800904776006D1C082DE6D3002C40F1D3
:10F4E0009F80002003A800210160002005E05FF05C
:10F4F000FF3102AA42F82010401C0028F7D0002457
:10F50000002559E002214AE04A48284490F850700A
:10F510003E00F6B236F0C0064648284490F9500046
:10F5200010F1010F47D002A93000FFF765FF002856
:10F5300041D0FFB2BF093000FFF775FF40B2FFF7BF
:10F5400078FF80464046002803D13800C0B2032827
:10F5500031D13800C0B2032803D103A93000FFF72E
:10F5600055FF3000FFF721FF814669463000FFF765
:10F5700043FF002803D04946C9B2022905D000281C
:10F5800019D14846C0B2032815D13800C0B20328AB
:10F590000AD15FFA89F9B9F1020FB3D10321C9B2D7
:10F5A0003000FFF7E2FE641C4046002803D039001B
:10F5B000C9B23000C0476D1C042DA5D32000C0B2D5
:10F5C000002829D0012501AA01210020FFF7FDFE16
:10F5D000002000E0401C002808D101A951F82010AB
:10F5E0006A4652F820209142F4D00025EDB2002D59
:10F5F00001D0002410E000200CE001A951F82010F7
:10F600006A4642F8201003A951F8201002AA42F8D5
:10F610002010401C0028F0D0E4B2002C7FF46FAF23
:10F6200005B0BDE8F08300000463004010650040B1
:10F630009C0F0300203D0020012210F01F018A4092
:10F64000664940B2400941F820207047020052B29A
:10F65000002A08D54901624A40B210F00F00104458
:10F6600000F8041C03E049015E4A40B2115470479F
:10F67000000B40B2704780B5C9B240B2FFF7E6FF59
:10F6800001BD80B540B2FFF7D7FF01BD0100080002
:10F6900040B2202290FBF2F0504A52F8200049B2CA
:10F6A000202291FBF2F302FB1311C84010F001007D
:10F6B00070474D490860704701215FF08042C0B239
:10F6C0001150704781B000215FF0804203001BB2EF
:10F6D000D1505FF0804100B208580090009801B00E
:10F6E00070475FF0804100B20858002801D0012027
:10F6F00000E00020C0B270473C49086070473C48B9
:10F700000068000C10F00100704710B506245FF08F
:10F710008040FFF7ADFF40B2FFF7B8FF00280FD1E0
:10F720005FF08040FFF7A4FF2100C9B240B2FFF7AD
:10F73000A2FF5FF08040FFF79BFF40B2FFF7A1FF01
:10F7400010BD020000202B490979002901D0852035
:10F7500007E028490A600121264A11710021254A43
:10F760005171704780B5FFF7D0FF0120FFF7C4FF4C
:10F7700001BD80B50C20FFF79FFFFFF7C0FF0028F9
:10F78000FBD101BD80B54FF48070FFF7AAFF0028C0
:10F7900011D04FF48070FFF795FF0120FFF789FF2C
:10F7A00014484079002806D10120124948710020F0
:10F7B0001049096888474FF48270FFF792FF0028CC
:10F7C0000AD04FF48270FFF77DFF0220FFF771FF30
:10F7D000012008490968884701BD000000E100E0F8
:10F7E00018ED00E000E400E00803004018050040C8
:10F7F0001804004078400020012210F01F018A40C8
:10F80000DFF8601140B2400941F82020704780B510
:10F81000FFF7AFFF0020DFF85011887001BD10B571
:10F82000002051480078002801D0852419E00020EC
:10F830004D49886000204C49486000204A490861D1
:10F8400000204949C8600FF28500FFF77AFF0400E5
:10F85000FBF7DBFC002801D1FFF784FF01204249C0
:10F860000870200010BD01000868002801D002685F
:10F870000A60704780B500208DF800006846FDF7EB
:10F8800015FD3948C068401E3749C8603648C06811
:10F89000002801D1FFF7BBFF9DF80000FDF70AFD2E
:10F8A00001BD38B504002000C0B2002801D1304DA0
:10F8B00005E02E4D03E02000C0B2496888472800CB
:10F8C000FFF7D1FF01000029F5D131BD10B50400CB
:10F8D0002000C0B2002805D1012023494870002033
:10F8E000FFF7DFFFE4B2012C05D101201E4988702B
:10F8F0000120FFF7D6FF10BD80B5002805D10120FB
:10F90000194948700020FFF7CCFF01BD80B5C0B297
:10F91000002804D0012806D003281DD021E00020B3
:10F92000FFF76AFF1DE000208DF800006846FDF734
:10F93000BDFC0D480078002801D1FFF770FF0A4890
:10F94000C068401C0849C8600120074988709DF8BC
:10F950000000FDF7AFFC04E0FFF704FFFFF78AFFAC
:10F96000FFE701BD80E100E0C03F0020D03F002064
:10F97000C83F002010B50446AFF30080204600F0D9
:10F9800005F80446AFF30080204610BD7CB500F1B9
:10F990000F06F608F600B04240D2082E04D2082620
:10F9A00002E0083000F047F8DFF804512C6821002D
:10F9B00005D1002007E00268B24221D2011D08688B
:10F9C0000028F8D12068291D0A68824222D01368D5
:10F9D000B34238BF111DF7D312E093190B60801B9F
:10F9E00054685C600B6818601660096800291DBFC8
:10F9F00048680028081D0020286002F1080076BD34
:10FA000061B10A681068A0F10803B342E5D25068FA
:10FA10000860EAE700F04EF80028C2D1002076BD69
:10FA200010B5040006D0AFF30080204600F003F8C4
:10FA3000AFF3008010BD002800D1704750B4A0F192
:10FA400008021368072B2BD913F0070F28D1184C85
:10FA5000616809B18A4202D25160626013E048686D
:10FA600000B3904238BF0146F9D31BE0964203D160
:10FA70001B180B600A4606E0486810B11344984210
:10FA80000ED350604A60506850B11368D11881425B
:10FA900006D1002121600168CB18136040685060D6
:10FAA00050BC704708680E18B242DFD250BC704795
:10FAB000884000200749086808B1002070470648C0
:10FAC000C008C00008600549C908C900091A0160DA
:10FAD000704700BFCC400020E7600020E08000209D
:10FAE00000000000180E030001000000CC07030016
:10FAF0000200000070060300030000005C0B03001E
:10FB000004000000700B030005000000840B0300DC
:10FB100006000000E809030007000000000A0300D7
:10FB200008000000180A030009000000140903007F
:10FB30000A000000300A03000B000000480A03001E
:10FB40000C000000980B03000D000000AC0B03003C
:10FB50000E000000E00C03000F000000C00B0300CB
:10FB600010000000600A030011000000F00C030008
:10FB700012000000780A030013000000D40B0300F9
:10FB8000800000009406030081000000300903009B
:10FB9000820000004C09030083000000EC07030012
:10FBA00084000000B806030085000000680503001B
:10FBB00086000000900A0300900000000C0803007B
:10FBC000910000002C08030092000000A80A030026
:10FBD000008200004C080300018200006809030055
:10FBE000028200008409030000840000DC06030098
:10FBF000018400003C05030002840000900503001E
:10FC000003840000000703002DE9F0410746884601
:10FC1000387810F0030F16461D4633D0384600F0F2
:10FC200099F878BBB8F1000F1CBFD8E9000186191C
:10FC3000012D2ED13888C10415D5396A07F1440247
:10FC4000384600F0A3F83A6B044602B93A69F968FD
:10FC5000384600F09BF8361B341A7A69F968384642
:10FC600000F094F8261A1EB94DB916F1010F09D00B
:10FC700097F903002A4631465FF0FF30064616F139
:10FC8000010F09D12320AFF300804FF0FF30BDE812
:10FC9000F081022DE8D1EBE7388810F4405F0ED0F8
:10FCA0007868F86038617861B8617868F86107F160
:10FCB0004400386207F13000786200203863B8F100
:10FCC000000F05D0D8E9020107F13402C2E90001B2
:10FCD00039884CF6FF60014039800020BDE8F08192
:10FCE00070B50546AFF300802888810415D56E688D
:10FCF0000024EA6895F903003146914212D2521A63
:10FD000000F04AF810F1010F1CBF00283618F0D19E
:10FD10000FE04DF6FF70014029802846AFF30080C8
:10FD2000002070BD0022002100F036F810F1010F14
:10FD300000D101246868E860A861E861002C298886
:10FD4000E7D041F4007129802846AFF300804FF0DE
:10FD5000FF3070BDF8B5A0B9AFF3008000250A4EA2
:10FD600008244FF0FF37306820B1FFF7B9FF0028B3
:10FD700048BF3D46361D641EF5D1AFF300802846CE
:10FD8000F2BDBDE8F240ABE77C2D0020914234BFCC
:10FD9000511A00210846704770B50C001500002666
:10FDA00004E02078F9F75CFB641C761CAE42F8D3C3
:10FDB000280070BD10B50446E068A169884251D39F
:10FDC000218849F202030B40022B08D008044CBFE3
:10FDD0004FF400704FF48440014321803BE001F474
:10FDE000C042B2F5C04F06D1A168884203D3204675
:10FDF000FFF7B0FF78BB208810F4406F02BF606847
:10FE000004F14401884217D14FF40070FFF7B2FDAE
:10FE1000606030B904F144006060E060401CA060A4
:10FE20000AE0218841F040012180E060606100F536
:10FE300000726068A260E06160682061A068A061F3
:10FE4000207841070AD502220021204600F00CF854
:10FE500010F1010F02D14FF0FF3010BD208840F4A7
:10FE6000C0402080002010BD70B504460D461646E7
:10FE7000AFF3008033462A4600212046FFF7C4FE38
:10FE800005462046AFF30080284670BD400D0300B4
:10FE900000000000580D0300000000003C0E0300AD
:10FEA00000000000700C030000000303900E03002C
:10FEB00000000000900F030000000303A00D0300EA
:10FEC00000000000180F030000000303DC0D030016
:10FED00000000303F40D0300000003030C0E0300F5
:10FEE00000000000200F030000000000280F0300A6
:10FEF00000000000A00F030000000000300F03000E
:10FF000000000000380F03000000000038B50400B6
:10FF10000ED0207810F0030F03D094F903000028CE
:10FF200009D5AFF30080204600F030F8AFF3008031
:10FF30004FF0FF3032BD2046FFF70CFF0546AFF310
:10FF400000802078410644BF606800F05DF8002022
:10FF5000606094F90300022804D90020C04608B16B
:10FF60004FF0FF35E06B48B10020C04608B14FF0BC
:10FF7000FF35E06B00F048F80020E063204600F019
:10FF800005F8AFF30080284632BDFEE701780A0687
:10FF900026D51C4A13680021834203D1002342F86E
:10FFA00021301BE05368012183421EBF0221936868
:10FFB0008342F3D0D368032183421EBF0421136917
:10FFC0008342EBD05369052183421EBF062193690A
:10FFD00083421EBF0721D3698342DFD000F014B8EB
:10FFE000002101804FF0FF31C17000F144014160F8
:10FFF000C160016141618161C161016200F1300153
:020000040003F7
:10000000416270477C2D0020FFF70ABD54686520CF
:1000100072657175657374656420636F6D62696E76
:100020006174696F6E206F6620545820616E642081
:100030005258207061636B6574206C656E677468DC
:100040007320697320746F6F206C6F6E6720627904
:10005000202575206D6963726F7365636F6E6473BD
:100060002E00000073645F626C655F6366675F7398
:10007000657428292072657475726E656420257315
:10008000207768656E20617474656D7074696E6741
:1000900020746F2073657420424C455F474154546F
:1000A000535F4346475F415454525F5441425F534C
:1000B000495A452E0000000073645F626C655F63FF
:1000C00066675F73657428292072657475726E6542
:1000D00064202573207768656E20617474656D7087
:1000E00074696E6720746F2073657420424C455F9D
:1000F00047415454535F4346475F53455256494323
:10010000455F4348414E4745442E000038B50C46F4
:10011000C5B22046AFF30080E068A169884204D3ED
:100120002046FFF747FE00280FD4E068401CE0603F
:1001300000F8015D2088010503D440050BD50A2D88
:1001400009D12046FFF706FE28B12046AFF3008014
:100150004FF0FF3032BD2046AFF30080284632BD5D
:1001600073645F626C655F6761705F646174615F37
:100170006C656E6774685F757064617465282920AA
:10018000287265717565737429206F6E20636F6EB8
:100190006E656374696F6E2030782578207265749F
:1001A00075726E65642025732E00000073645F62B3
:1001B0006C655F6366675F73657428292072657478
:1001C00075726E6564202573207768656E20617492
:1001D00074656D7074696E6720746F207365742028
:1001E000424C455F4741505F4346475F524F4C4545
:1001F0005F434F554E542E0073645F626C655F63BE
:1002000066675F73657428292072657475726E6500
:1002100064202573207768656E20617474656D7045
:1002200074696E6720746F2073657420424C455F5B
:10023000434F4D4D4F4E5F4346475F56535F5555B5
:1002400049442E0073645F626C655F6366675F7329
:10025000657428292072657475726E656420257333
:10026000207768656E20617474656D7074696E675F
:1002700020746F2073657420424C455F434F4E4E8F
:100280005F4346475F4741502E00000073645F6242
:100290006C655F6366675F73657428292072657497
:1002A00075726E6564202573207768656E206174B1
:1002B00074656D7074696E6720746F207365742047
:1002C000424C455F434F4E4E5F4346475F47415464
:1002D000542E000080687047F8B568464BDF002850
:1002E00004D10D4901A8FDF7A8FD0FE0052801D0B4
:1002F000F8F71EFF05B000BD01A8FFF7EBFF02688D
:1003000041680098904701A8FDF79EFD01A8FFF7FE
:10031000E1FF0028E1D0EFE7000E0300513753540E
:1003200066696A6768775A306E5770715573494AC3
:10033000364C4142797A44434533474875345978BD
:100340004D39504F6164386272566F586B6C6D3125
:10035000324676354B52634E74652B2F00000000F9
:1003600054686520726571756573746564205458AE
:100370002F5258207061636B6574206C656E6774D2
:100380006820697320746F6F206C6F6E67206279CC
:100390002025752F2575206F63746574732E0000FA
:1003A00019E050F8042BD30744BFA9F101039A18B0
:1003B000091F0023042942F8043BF9D25FEA817C3B
:1003C000134604D54FF0000CA2F800C09B1CC907CF
:1003D00044BF0021197050F8041B0029E1D1704777
:1003E00038B50D4D0824286800281CBF017811F08D
:1003F000030F05D090F90310002958BFFFF786FDC1
:100400002D1D641EEFD1BDE83840002200214FF0C1
:10041000FF30FFF7C1BC00BF7C2D002073645F621A
:100420006C655F67617474635F65786368616E674C
:10043000655F6D74755F72657175657374282920C9
:1004400072657475726E65642025732E000000005D
:100450004368616E6765207468652052414D207362
:1004600074617274206C6F636174696F6E20667260
:100470006F6D203078257820746F20307825782EA5
:100480000000000073645F626C655F676174747381
:100490005F65786368616E67655F6D74755F7265CF
:1004A000706C7928292072657475726E65642025D8
:1004B000732E0000496E73756666696369656E74B4
:1004C0002052414D20616C6C6F63617465642066DD
:1004D0006F722074686520536F6674446576696333
:1004E000652E00004661696C65642072656365690C
:1004F00076696E67204E5553206D6573736167652D
:100500002E204572726F7220307825782E200000E0
:100510004D6178696D756D2052414D2073697A6522
:1005200020666F72206170706C69636174696F6EB0
:1005300020697320307825782E0000004E52465FE7
:100540004552524F525F424C455F495053505F43B2
:1005500048414E4E454C5F414C52454144595F45E0
:1005600058495354530000004E52465F4552524F73
:10057000525F4D4F44554C455F414C5245414459A3
:100580005F494E495449414C495A454400000000D6
:100590004E52465F4552524F525F424C455F495062
:1005A00053505F4C494E4B5F444953434F4E4E4569
:1005B000435445440000000010B507497944183100
:1005C000064C7C44163404E00A68081D1144884730
:1005D0000146A142F8D110BD700100008C0100005D
:1005E00052544320696E7374616E636520616C724E
:1005F0006561647920696E697469616C697A6564A2
:100600002E000000425420496E666F726D6174695D
:100610006F6E2D2D2D2D2D2D2D2D2D2D2D2D2D2D87
:100620002D2D0D0A000000002D2D2D2D2D2D2D2DF1
:100630002D2D2D2D2D2D2D2D2D2D2D2D2D2D2D2DEA
:100640002D2D2D2D2D2D0D0A0D0A0000666C7368C1
:1006500020726561643A20307825782030782578DA
:1006600020307825782030782578200D0A00000089
:100670004E52465F4552524F525F534F4654444587
:10068000564943455F4E4F545F454E41424C4544A9
:10069000000000004E52465F4552524F525F4D4F90
:1006A00044554C455F4E4F545F494E495449414C67
:1006B000495A4544000000004E52465F4552524F91
:1006C000525F4D555445585F434F4E445F494E4924
:1006D000545F4641494C4544000000004E52465F7D
:1006E0004552524F525F424C455F495053505F5202
:1006F000585F504B545F5452554E4341544544004B
:100700004E52465F4552524F525F424C455F4950F0
:1007100053505F504545525F52454A454354454406
:10072000000000004EF68851CEF20001086840F447
:1007300070000860BFF34F8FBFF36F8F4FF00070F2
:10074000E1EE100A7047000059FCFFFF4013000063
:10075000A02D0020000000003F6AFFFF6808000095
:1007600030020000D82A0020FEE70000FFFFFFFF54
:10077000FFFFFFFFFFFFFFFFFFFFFFFF0000000085
:10078000000000000000D6010601000073645F62F3
:100790006C655F656E61626C652829207265747591
:1007A000726E65642025732E00000000480F030060
:1007B000500F03006C0803008C080300200D030099
:1007C000300D0300500F0300580F03004E52465FD8
:1007D0004552524F525F5356435F48414E444C4539
:1007E000525F4D495353494E470000004E52465FF9
:1007F0004552524F525F4D555445585F554E4C4FE0
:10080000434B5F4641494C45440000004E52465F11
:100810004552524F525F4150495F4E4F545F494DD0
:10082000504C454D454E5445440000004E52465FE5
:100830004552524F525F464541545552455F4E4FC7
:10084000545F454E41424C45440000004E52465FC5
:100850004552524F525F4452565F5457495F45527A
:10086000525F4F56455252554E0000007DA4020083
:100870000000000067AA02000000000059B8020052
:10088000AC3F0020EBAF0200A02D00200120C046AD
:10089000002801D0FFF790FEAFF300800020AFF3F7
:1008A0000080F8F714F900F000F800F001B8FEE756
:1008B0000746FFF795FD3846F7F774FBFBE7FEE7C1
:1008C00044617461206C656E2069732073657420C7
:1008D000746F20307825582825642900425420560A
:1008E00065723D2573202D2D2D2D2D2D2D2D2D2D7A
:1008F0002D2D720A000000000D0A424C4520554182
:1009000052542073746172746564202121212D2D4D
:100910002D0D0A004E52465F4552524F525F494ECE
:1009200056414C49445F4C454E4754480000000036
:100930004E52465F4552524F525F4D555445585F97
:10094000494E49545F4641494C4544004E52465F2A
:100950004552524F525F4D555445585F4C4F434B93
:100960005F4641494C4544004E52465F4552524F06
:10097000525F4452565F5457495F4552525F414E51
:1009800041434B004E52465F4552524F525F4452D4
:10099000565F5457495F4552525F444E41434B00A6
:1009A0001A0000001C000000050000000700000005
:1009B0000000000000E0D70125734C6F67732064CE
:1009C000726F70706564202825642925730D0A00F4
:1009D0000000000000000000000000000000000017
:1009E00000000000000000004E52465F4552524F8A
:1009F000525F4E4F545F535550504F525445440030
:100A00004E52465F4552524F525F494E56414C49F5
:100A1000445F504152414D004E52465F4552524F45
:100A2000525F494E56414C49445F5354415445002E
:100A30004E52465F4552524F525F494E56414C49C5
:100A4000445F464C414753004E52465F4552524F19
:100A5000525F494E56414C49445F44415441000065
:100A60004E52465F4552524F525F494E56414C4995
:100A7000445F4144445200004E52465F4552524F3B
:100A8000525F434F4E4E5F434F554E54000000009F
:100A90004E52465F4552524F525F53544F52414758
:100AA000455F46554C4C00004E52465F4552524FF2
:100AB000525F494F5F50454E44494E470000000089
:100AC00038B504460D46284600F006F8A84218BF7F
:100AD0000024204632BDFEE70149FFF717BB00BFE7
:100AE000EC2C00205254433A20696E697469616CA1
:100AF000697A65642E000000566572303130345FCB
:100B0000323032323131313600000000416E6472D1
:100B10006F69647E7E7E7E7E0D0A0D0A00000000F5
:100B2000424C4520436F6E6E65637465642E0D0AFA
:100B300000000000446576696365204E616D6520A4
:100B40003A202573200D0A004261636B656E647361
:100B500020666C7573686564000000004E52465F45
:100B60004552524F525F494E5445524E414C00003F
:100B70004E52465F4552524F525F4E4F5F4D454D6C
:100B8000000000004E52465F4552524F525F4E4F9A
:100B9000545F464F554E44004E52465F4552524FA9
:100BA000525F444154415F53495A45004E52465F9B
:100BB0004552524F525F54494D454F555400000025
:100BC0004E52465F4552524F525F464F5242494441
:100BD00044454E004E52465F4552524F525F524579
:100BE000534F555243455300556E6B6E6F776E20D1
:100BF0006572726F7220636F646500007040002040
:100C00006840002070400020EC3A002018000000EE
:100C100053797374656D207265736574000000000C
:100C20009ECADC240EE5A9E093F3A3B50000406E54
:100C3000446973636F6E6E656374656400000000E1
:100C40004254205665723D2573202D2D2D0D0A002E
:100C500053697465203A202573200D0A00000000B6
:100C6000557365724944203A202573200D0A00000F
:100C70006E72665F626C655F67617474000000008D
:100C800030313233343536373839414243444546C2
:100C90007274745F6C6F675F6261636B656E640032
:100CA0000000000000000000000000000000000044
:100CB000600F0300680F0300000000000000000048
:100CC000300D0300400D0300000000000000000094
:100CD000580F0300600F0300000000000000000038
:100CE0004E52465F4552524F525F4E554C4C00009B
:100CF0004E52465F4552524F525F42555359000083
:100D000001488047014800472FED0200310E0300E3
:100D10007C0D030000000000900C0300E02B00207D
:100D2000579F0200002B0020859D02002C400020D0
:100D3000B5B4020000000000D9020300000000006A
:100D40006170705F627574746F6E000046617461EB
:100D50006C206572726F72006170705F74696D658E
:100D6000720000000000000090400020398D020059
:100D7000436F6E6E656374656400000045DF0200BA
:100D800067DF020065DF0200AC3B00207F0000004F
:100D9000803F00203C25733E2025733A2000000050
:100DA0007077725F6D676D7400000000D0090300FA
:100DB000E809030004000000A00C0300B00C0300CD
:100DC00008000000B00C0300C00C03000800000085
:100DD000C00C0300D00C0300080000006E72665FB8
:100DE0007364685F626C6500AC070300CC070300A6
:100DF000080000006E72665F7364685F736F630063
:100E0000D00C0300E00C030008000000736F727444
:100E10006C697374000000004E52465F53554343A3
:100E2000455353005465726D696E616C000000009B
:100E3000AFF30080FFF776FCFFF728FD626C655F7B
:100E40006E7573000000000000000000000000004C
:100E50000338FDD87047000025730A282573290040
:100E60000338FDD8704700000000000000000000BB
:100E70000000000000000000770A000000000000F1
:100E8000770A0000000000007ADA0000000000008D
:100E9000636C6F636B000000000000000000000046
:100EA0000338FDD8704700006572726F7200000051
:100EB0007761726E696E6700696E666F0000000090
:100EC00064656275670000001B5B306D0000000008
:100ED0001B5B313B33306D001B5B313B33316D00AD
:100EE0001B5B313B33326D001B5B313B33336D0099
:100EF0001B5B313B33346D001B5B313B33356D0085
:100F00001B5B313B33366D001B5B313B33376D0070
:100F100020253032780000006E72665F73646800CE
:100F2000434C4F434B0000004750494F544500008D
:100F300055415254000000005541525445000000F4
:100F40005345474745520000A1E102000000000060
:100F50007585020000000000F9F8020000000000A2
:100F60000DF902000000000000002E004300FEE723
:100F7000D43F002001000600111213140D0E0F10B3
:100F8000403F0020603F0020000000000000000003
:100F90006170700002000005D82A00200000005097
:100FA00050525300CDCD0200A7C60200FEE7FEE777
:100FB000FEE7FEE7FEE7FEE7FEE7FEE7FEE7FEE709
:100FC000FEE7FEE73006001001401100040001308A
:100FD000012000400951086007F80A0300A84000FA
:100FE000200120D10113F82A2A1101F0092801005B
:100FF000020053465F30303100011140F0012948B2
:10100000510001F0040973667573657241F00809B7
:10101000706173733235383021212452FF1B100365
:10102000A80E0300B00412B80412C00412C80412BF
:10103000D00412D80412E00412E80412F00412F8EA
:10104000041003000F0300080410030090D003688D
:1010500008F1070452FF01F2006A14100100006C4D
:101060000C12017C47242C5030011772028A121195
:1010700008522D0C521508610152ED1012DB085276
:10108000011A1601A712E84412E90452E804211BD0
:10109000A10852D40CF10B01100702040101243EF7
:1010A0000020740452240421346108F00412302D0D
:1010B00000201C2D484003080202D43D4021082195
:1010C0000421346108127844F212644812A4B41264
:0C10D000EC04F206342C0002FFFF1400B8
:0400000500030E31B5
:00000001FF
